:020000040000FA
:0408000098EF0BF072
:1008100003B275EF05F0F2B493EF05F09EB09BEFD5
:1008200005F09EB2A3EF05F0F2A81AEF04F0F2B2C1
:1008300023EF04F0F2B01FEF04F047EF0BF0F29655
:10084000F29047EF0BF0CD90F2929EA02DEF04F0C6
:100850000101533F2DEF04F0542BB2C1B6F1B3C1E7
:10086000B7F1B4C1B8F1B5C1B9F1AEC1B2F1AFC120
:10087000B3F1B0C1B4F1B1C1B5F1AAC1AEF1ABC130
:10088000AFF1ACC1B0F1ADC1B1F1A6C1AAF1A7C140
:10089000ABF1A8C1ACF1A9C1ADF1A2C1A6F1A3C150
:1008A000A7F1A4C1A8F1A5C1A9F19EC1A2F19FC160
:1008B000A3F1A0C1A4F1A1C1A5F19AC19EF19BC170
:1008C0009FF19CC1A0F19DC1A1F1CECF9AF1CFCFF4
:1008D0009BF153C19CF154C19DF1CF6ACE6A0101D5
:1008E000536B546B9E90CD800FBC0F8E0FBA7CEF74
:1008F00004F00F8A47EF0BF013880F8C0FBEB9EF8F
:1009000004F09AC19EF19BC19FF19CC1A0F19DC1D1
:10091000A1F19EC1A2F19FC1A3F1A0C1A4F1A1C107
:10092000A5F1A2C1A6F1A3C1A7F1A4C1A8F1A5C1D7
:10093000A9F1A6C1AAF1A7C1ABF1A8C1ACF1A9C1A7
:10094000ADF1AAC1AEF1ABC1AFF1ACC1B0F1ADC177
:10095000B1F1AEC1B2F1AFC1B3F1B0C1B4F1B1C147
:10096000B5F1B2C1B6F1B3C1B7F1B4C1B8F1B5C117
:10097000B9F101015E6B5F6B606B616B9A515E2731
:100980009B515F239C5160239D5161239E515E27A3
:100990009F515F23A0516023A1516123A2515E2783
:1009A000A3515F23A4516023A5516123A6515E2763
:1009B000A7515F23A8516023A9516123AA515E2743
:1009C000AB515F23AC516023AD516123AE515E2723
:1009D000AF515F23B0516023B1516123B2515E2703
:1009E000B3515F23B4516023B5516123B6515E27E3
:1009F000B7515F23B8516023B9516123D8900101E9
:100A0000613360335F335E33D8900101613360330B
:100A10005F335E33D8900101613360335F335E33FF
:100A200000C10CF101C10DF102C10EF103C10FF1C2
:100A300004C110F105C111F106C112F107C113F192
:100A400008C114F109C115F10AC116F10BC117F162
:100A500034C135F111B838EF05F00101620E046FB1
:100A6000010E056F000E066F000E076F41EF05F0D7
:100A70000101A70E046F020E056F000E066F000E37
:100A8000076F5EC100F15FC101F160C102F161C198
:100A900003F183EC2FF003BF04D01CBE02D01CA0D6
:100AA000108C11A059EF05F010BA59EF05F00F8026
:100AB000108A0CC100F10DC101F10EC102F10FC18C
:100AC00003F110C104F111C105F112C106F113C106
:100AD00007F114C108F115C109F116C10AF117C1D6
:100AE0000BF135C134F147EF0BF00392ABB2AB9889
:100AF000AB88030103EE00F080517F0BE92604C0B0
:100B0000EFFF802B8151805D700BD8A48B82000099
:100B10008051815D700BD8A48B9281518019D8B41B
:100B2000079047EF0BF0F2940101453F47EF0BF0C0
:100B3000462B47EF0BF09E900101533F47EF0BF020
:100B4000542B47EF0BF09E9211B843EF08F00400CE
:100B500066A1ABEF05F08BB4B5EF05F010ACB5EFC7
:100B600005F08B84109CB6EF05F08B94077C07ACE6
:100B7000D1EF05F0C274C2B4CBEF05F0C3CFB7F527
:100B8000C4CFB8F50501D890B833B733D890B8338F
:100B9000B733D2EF05F0C3CF55F1C4CF56F1D2EF42
:100BA00005F0C28207B444EF06F047C14BF148C1DB
:100BB0004CF149C14DF14AC14EF15EC162F15FC1D4
:100BC00063F160C164F161C165F113A8EAEF05F05A
:100BD000138C13989AC1BAF19BC1BBF19CC1BCF1B3
:100BE0009DC1BDF19EC1BEF19FC1BFF1A0C1C0F1C9
:100BF000A1C1C1F1A2C1C2F1A3C1C3F1A4C1C4F199
:100C0000A5C1C5F1A6C1C6F1A7C1C7F1A8C1C8F168
:100C1000A9C1C9F1AAC1CAF1ABC1CBF1ACC1CCF138
:100C2000ADC1CDF1AEC1CEF1AFC1CFF1B0C1D0F108
:100C3000B1C1D1F1B2C1D2F1B3C1D3F1B4C1D4F1D8
:100C4000B5C1D5F1B6C1D6F1B7C1D7F1B8C1D8F1A8
:100C5000B9C1D9F1B7C5B9F5B8C5BAF5B9C5BBF5CC
:100C6000BAC5BCF5010155515B2756515C23E86AB2
:100C70005D230E2E44EF06F05CC157F15DC158F1C3
:100C80005B6B5C6B5D6B078E0201002F47EF0BF017
:100C90003C0E006F1D50E00BE00AE86612881BBE98
:100CA00002D01BB4108E00C10CF101C10DF102C1C4
:100CB0000EF103C10FF104C110F105C111F106C11C
:100CC00012F107C113F108C114F109C115F10AC1EC
:100CD00016F10BC117F134C135F181AAACEF06F062
:100CE00015A4F7EF06F005012F51000AD8B43AEF2A
:100CF00007F005012F51010AD8B4B6EF06F005013F
:100D00002F51020AD8B4F7EF06F005012F51030A5C
:100D1000D8B4F7EF06F005012F51040AD8B4F7EF65
:100D200006F005012F51050AD8B4F7EF06F00501CA
:100D30002F51060AD8B4F7EF06F005012F51070A24
:100D4000D8B4F7EF06F005012F51320AD8B4B4EF4A
:100D500006F02F6B3AEF07F000011650030AD8B4E3
:100D6000F7EF06F03AEF07F03AEF07F005015767A3
:100D7000C1EF06F05867C1EF06F05967C1EF06F002
:100D80005A67C5EF06F03AEF07F05BC500F15CC5A6
:100D900001F15DC502F15EC503F10101010E046FB1
:100DA000000E056F000E066F000E076F83EC2FF02C
:100DB00000C15BF501C15CF502C15DF503C15EF5E3
:100DC00001010067EBEF06F00167EBEF06F0026749
:100DD000EBEF06F003673AEF07F057C55BF558C530
:100DE0005CF559C55DF55AC55EF524EF07F00FBEF9
:100DF0000CEF07F010A011EF07F00101476708EFB3
:100E000007F0486708EF07F0496708EF07F04A67FF
:100E10000CEF07F011EF07F007AE11EF07F024EF2A
:100E200007F00501312F3AEF07F03C0E316F302FFC
:100E30003AEF07F00101000E626FE00E636FA50E3E
:100E4000646F010E656F138800011650000AD8B454
:100E500032EF07F000011650030AD8B437EF07F05D
:100E60003AEF07F00001010E166E3AEF07F00001AD
:100E7000040E166E0501666B37B740EF07F066810A
:100E80000CC100F10DC101F10EC102F10FC103F15E
:100E900010C104F111C105F112C106F113C107F12E
:100EA00014C108F115C109F116C10AF117C10BF1FE
:100EB00035C134F100C10CF101C10DF102C10EF1D7
:100EC00003C10FF104C110F105C111F106C112F106
:100ED00007C113F108C114F109C115F10AC116F1D6
:100EE0000BC117F134C135F101018E677FEF07F0B7
:100EF0008F677FEF07F090677FEF07F0916783EFD1
:100F000007F0B4EF07F092C100F193C101F194C171
:100F100002F195C103F10101010E046F000E056F8E
:100F2000000E066F000E076F83EC2FF000C192F1E8
:100F300001C193F102C194F103C195F10101006770
:100F4000A9EF07F00167A9EF07F00267A9EF07F023
:100F50000367B4EF07F08EC192F18FC193F190C196
:100F600094F191C195F10F80D57ED5BE6ED0D6CFCC
:100F700047F1D7CF48F145C149F1E86AE8CF4AF1D6
:100F8000138A1CBE02D01CA0108C109047C100F127
:100F900048C101F149C102F14AC103F101010A0E40
:100FA000046F000E056F000E066F000E076F83ECD6
:100FB0002FF003AF1080010154A7EBEF07F00F9A59
:100FC0000F9C0F9E0101000E5E6F600E5F6F3D0E65
:100FD000606F080E616F010147BFFBEF07F04867C4
:100FE000FBEF07F04967FBEF07F04A67FBEF07F0FD
:100FF000F28820EF08F0F2985E6B5F6B606B616BBC
:101000009A6B9B6B9C6B9D6B9E6B9F6BA06BA16B9C
:10101000A26BA36BA46BA56BA66BA76BA86BA96B4C
:10102000AA6BAB6BAC6BAD6BAE6BAF6BB06BB16BFC
:10103000B26BB36BB46BB56BB66BB76BB86BB96BAC
:10104000D76AD66A0101456B466B0CC100F10DC130
:1010500001F10EC102F10FC103F110C104F111C180
:1010600005F112C106F113C107F114C108F115C150
:1010700009F116C10AF117C10BF135C134F147EF7F
:101080000BF047EF0BF00201002FABEF0AF0D59EFB
:10109000D6CF47F1D7CF48F145C149F1E86AE8CF4B
:1010A0004AF1138AD76AD66A0101456B466BD58E21
:1010B0001D50E00BE00AE86612881BBE02D01BB48C
:1010C000108E1AAE1F8C00C10CF101C10DF102C1CE
:1010D0000EF103C10FF104C110F105C111F106C1F8
:1010E00012F107C113F108C114F109C115F10AC1C8
:1010F00016F10BC117F134C135F10FA0109A11B8D8
:101100008DEF08F00101620E046F010E056F000EF5
:10111000066F000E076F96EF08F00101A70E046F2F
:10112000020E056F000E066F000E076F47C100F13B
:1011300048C101F149C102F14AC103F183EC2FF02A
:1011400003BFA9EF08F01CBE02D01CA0108C11B088
:101150000F800CC100F10DC101F10EC102F10FC1F0
:1011600003F110C104F111C105F112C106F113C15F
:1011700007F114C108F115C109F116C10AF117C12F
:101180000BF135C134F102013C0E006F00C10CF1CE
:1011900001C10DF102C10EF103C10FF104C110F143
:1011A00005C111F106C112F107C113F108C114F113
:1011B00009C115F10AC116F10BC117F134C135F19E
:1011C00081BAE6EF08F015B225EF09F015A025EF7A
:1011D00009F015A470EF09F005012F51000AD8B4E9
:1011E000B3EF09F005012F51010AD8B42FEF09F030
:1011F00005012F51020AD8B470EF09F005012F51F3
:10120000030AD8B470EF09F005012F51040AD8B4CD
:1012100070EF09F005012F51050AD8B470EF09F0FD
:1012200005012F51060AD8B470EF09F005012F51BE
:10123000070AD8B470EF09F005012F51320AD8B46B
:101240002DEF09F02F6BB3EF09F000011650030AE0
:10125000D8B470EF09F0B3EF09F0B3EF09F005016E
:1012600057673AEF09F058673AEF09F059673AEFD4
:1012700009F05A673EEF09F0B3EF09F05BC500F1E2
:101280005CC501F15DC502F15EC503F10101010E0E
:10129000046F000E056F000E066F000E076F83ECE3
:1012A0002FF000C15BF501C15CF502C15DF503C122
:1012B0005EF50101006764EF09F0016764EF09F072
:1012C000026764EF09F00367B3EF09F057C55BF5F8
:1012D00058C55CF559C55DF55AC55EF59DEF09F039
:1012E0000FBE85EF09F010A08AEF09F001014767F2
:1012F00081EF09F0486781EF09F0496781EF09F054
:101300004A6785EF09F08AEF09F007AE8AEF09F026
:101310009DEF09F00501312FB3EF09F03C0E316F5D
:10132000302FB3EF09F00101000E626FE00E636F22
:10133000A50E646F010E656F138800011650000A38
:10134000D8B4ABEF09F000011650030AD8B4B0EFDF
:1013500009F0B3EF09F00001010E166EB3EF09F0CA
:101360000001040E166E0501666B37B7B9EF09F080
:1013700066810CC100F10DC101F10EC102F10FC176
:1013800003F110C104F111C105F112C106F113C13D
:1013900007F114C108F115C109F116C10AF117C10D
:1013A0000BF135C134F100C10CF101C10DF102C1E5
:1013B0000EF103C10FF104C110F105C111F106C115
:1013C00012F107C113F108C114F109C115F10AC1E5
:1013D00016F10BC117F134C135F101018E67F8EF39
:1013E00009F08F67F8EF09F09067F8EF09F091675F
:1013F000FCEF09F02DEF0AF092C100F193C101F169
:1014000094C102F195C103F10101010E046F000EB8
:10141000056F000E066F000E076F83EC2FF000C102
:1014200092F101C193F102C194F103C195F101015F
:10143000006722EF0AF0016722EF0AF0026722EF4D
:101440000AF003672DEF0AF08EC192F18FC193F17C
:1014500090C194F191C195F10F80109047C100F1B6
:1014600048C101F149C102F14AC103F101010A0E6B
:10147000046F000E056F000E066F000E076F83EC01
:101480002FF003AF1080010154A753EF0AF00F9A19
:101490000F9C0F9E0101000E5E6F600E5F6F3D0E90
:1014A000606F080E616F47C100F148C101F149C189
:1014B00002F14AC103F10101140E046F050E056F1C
:1014C000000E066F000E076F83EC2FF003AF6CEF7A
:1014D0000AF0F28891EF0AF0F2985E6B5F6B606B36
:1014E000616B9A6B9B6B9C6B9D6B9E6B9F6BA06BF8
:1014F000A16BA26BA36BA46BA56BA66BA76BA86B70
:10150000A96BAA6BAB6BAC6BAD6BAE6BAF6BB06B1F
:10151000B16BB26BB36BB46BB56BB66BB76BB86BCF
:10152000B96B0CC100F10DC101F10EC102F10FC187
:1015300003F110C104F111C105F112C106F113C18B
:1015400007F114C108F115C109F116C10AF117C15B
:101550000BF135C134F104008BB4B6EF0AF010ACD6
:10156000B6EF0AF08B84109CB7EF0AF08B94077CDF
:1015700007ACD2EF0AF0C274C2B4CCEF0AF0C3CF0A
:10158000B7F5C4CFB8F50501D890B833B733D890C4
:10159000B833B733D3EF0AF0C3CF55F1C4CF56F108
:1015A000D3EF0AF0C28207B445EF0BF047C14BF10D
:1015B00048C14CF149C14DF14AC14EF15EC162F1E1
:1015C0005FC163F160C164F161C165F113A8EBEF24
:1015D0000AF0138C13989AC1BAF19BC1BBF19CC15C
:1015E000BCF19DC1BDF19EC1BEF19FC1BFF1A0C1C3
:1015F000C0F1A1C1C1F1A2C1C2F1A3C1C3F1A4C193
:10160000C4F1A5C1C5F1A6C1C6F1A7C1C7F1A8C162
:10161000C8F1A9C1C9F1AAC1CAF1ABC1CBF1ACC132
:10162000CCF1ADC1CDF1AEC1CEF1AFC1CFF1B0C102
:10163000D0F1B1C1D1F1B2C1D2F1B3C1D3F1B4C1D2
:10164000D4F1B5C1D5F1B6C1D6F1B7C1D7F1B8C1A2
:10165000D8F1B9C1D9F1B7C5B9F5B8C5BAF5B9C5A9
:10166000BBF5BAC5BCF5010155515B2756515C234A
:10167000E86A5D230E2E45EF0BF05CC157F15DC1AA
:1016800058F15B6B5C6B5D6B078E47EF0BF002C034
:10169000E0FF005001C0D8FF1000A6B24DEF0BF0E4
:1016A0000CC0A9FF0BC0A8FFA69EA69CA684F29E14
:1016B000550EA76EAA0EA76EA682F28EA694A6B2AB
:1016C0005FEF0BF00C2A1200A96EA69EA69CA680C6
:1016D000A8500C2A120004012C0E826F94EC0EF01C
:1016E00098EC30F00C5064EC0BF0E8CF00F10C50AB
:1016F00064EC0BF0E8CF01F101AF84EF0BF00101D6
:10170000FF0E026FFF0E036F21EC30F0296790EFA0
:101710000BF00401200E826F94EC0EF095EF0BF0AD
:1017200004012D0E826F94EC0EF02BEC2EF01200C3
:1017300015941596076A0F6A106A116A126A136A7D
:10174000166A0F010D0EC16E860EC06E030EC26EBC
:101750000F01680E896E130E926E080E8A6EF30EDC
:10176000936E8B6A900E946EC80E64EC0BF0E8CF0B
:10177000E8FF1098E8A0108810A805D00E0E256E7E
:101780008E0E266E04D00F0E256E8F0E266E30EC58
:1017900031F0F18EF19EFC0E64EC0BF0E8CF0BF013
:1017A0000BA011800BA211820BA411840BA811882D
:1017B000C90E64EC0BF0E8CF1AF0CA0E64EC0BF023
:1017C000E8CF1BF0CB0E64EC0BF0E8CF1CF0CC0E96
:1017D00064EC0BF0E8CF1DF0FB0E64EC0BF0E8CFEF
:1017E00037F0CE0E64EC0BF0E8CF14F0CD0E64ECC5
:1017F0000BF0E8CF36F01F6A206A0E6A01015B6BBE
:101800005C6B5D6B576B586BF29A0101476B486BD1
:10181000496B4A6B4B6B4C6B4D6B4E6B4F6B506B0C
:10182000516B526B456B466BD76AD66A0F01280E17
:10183000D56EF28A9D90B00ECD6E01015E6B5F6B2E
:10184000606B616B626B636B646B656B666B676B24
:10185000686B696B536B546BCF6ACE6A0F9A0F9C9F
:101860000F9E9D80760ECA6E9D8202013C0E006F17
:10187000CC6A160E64EC0BF0E8CF00F1170E64ECA6
:101880000BF0E8CF01F1180E64EC0BF0E8CF02F199
:10189000190E64EC0BF0E8CF03F1010103AF6BEF1D
:1018A0000CF098EC30F0160E0C6E00C10BF04DEC05
:1018B0000BF0170E0C6E01C10BF04DEC0BF0180E77
:1018C0000C6E02C10BF04DEC0BF0190E0C6E03C147
:1018D0000BF04DEC0BF000C18EF101C18FF102C194
:1018E00090F103C191F100C192F101C193F102C1E4
:1018F00094F103C195F11A0E64EC0BF0E8CF00F1FE
:101900001B0E64EC0BF0E8CF01F11C0E64EC0BF045
:10191000E8CF02F11D0E64EC0BF0E8CF03F10101FA
:1019200003AFC1EF0CF098EC30F01A0E0C6E00C152
:101930000BF04DEC0BF01B0E0C6E01C10BF04DECDF
:101940000BF01C0E0C6E02C10BF04DEC0BF01D0EDB
:101950000C6E03C10BF04DEC0BF01A0E64EC0BF0A7
:10196000E8CF00F11B0E64EC0BF0E8CF01F11C0E88
:1019700064EC0BF0E8CF02F11D0E64EC0BF0E8CF45
:1019800003F100C196F101C197F102C198F103C1C1
:1019900099F1240EAC6E900EAB6E240EAC6E080E58
:1019A000B86E000EB06E1F0EAF6E0401806B816BBF
:1019B0000F01900EAB6E0F019D8A0301806B816B4E
:1019C000C26B8B92D5EC35F0D5EC35F0B7EC37F037
:1019D000B3EC33F0200E64EC0BF0E8CF2FF50501EB
:1019E0002F51FF0AD8A4FCEF0CF02F6B200E0C6EC9
:1019F0002FC50BF04DEC0BF00501010E306F3C0EC6
:101A0000316F250E64EC0BF0E8CF00F1260E64EC8C
:101A10000BF0E8CF01F1270E64EC0BF0E8CF02F1F8
:101A2000280E64EC0BF0E8CF03F1010103AF33EFB4
:101A30000DF098EC30F0250E0C6E00C10BF04DEC63
:101A40000BF0260E0C6E01C10BF04DEC0BF0270EC7
:101A50000C6E02C10BF04DEC0BF0280E0C6E03C1A6
:101A60000BF04DEC0BF000C157F501C158F502C168
:101A700059F503C15AF500C15BF501C15CF502C11E
:101A80005DF503C15EF5290E64EC0BF0E8CF5FF560
:101A9000050160515F5DD8A05FC560F5210E64EC63
:101AA0000BF0E8CF00F1220E64EC0BF0E8CF01F16F
:101AB000230E64EC0BF0E8CF02F1240E64EC0BF083
:101AC000E8CF03F1010103AF94EF0DF098EC30F093
:101AD000210E0C6E00C10BF04DEC0BF0220E0C6EC3
:101AE00001C10BF04DEC0BF0230E0C6E02C10BF09C
:101AF0004DEC0BF0240E0C6E03C10BF04DEC0BF013
:101B0000210E64EC0BF0E8CF00F1220E64EC0BF038
:101B1000E8CF01F1230E64EC0BF0E8CF02F1240EC4
:101B200064EC0BF0E8CF03F100C161F501C162F58F
:101B300002C163F503C164F5FBEC32F0E1EC31F076
:101B400039EC31F01590C70E64EC0BF0E8CF00F1E2
:101B5000010100B1AFEF0DF01592B0EF0DF015825D
:101B600081AABEEF0DF015B4B9EF0DF01580BEEFF0
:101B70000DF0F6EC37F015A05DEF38F0079000019E
:101B8000F28EF28C12AE03D012BC6CEF19F007B0DB
:101B9000AAEF2CF00FB0A6EF25F010BEA6EF25F0AF
:101BA00012B8A6EF25F000011650010AD8B49FEF35
:101BB0001DF081BAE4EF0DF000011650040AD8B40C
:101BC00018EF1CF0EAEF0DF000011650040AD8B42B
:101BD000DBEF1DF00301805181197F0BD8B4AAEF10
:101BE0002CF013EE00F081517F0BE126812BE7CF23
:101BF000E8FFE00BD8B4AAEF2CF023EE82F0C2513C
:101C00003F0BD926E7CFDFFFC22BDF50780AD8A4DD
:101C1000AAEF2CF0078092C100F193C101F194C1A9
:101C200002F195C103F10101040E046F000E056F6E
:101C3000000E066F000E076F83EC2FF000AF2AEF47
:101C40000EF00101030E926F000E936F000E946F61
:101C5000000E956F03018251720AD8B427EF25F068
:101C60008251520AD8B427EF25F08251750AD8B4B0
:101C700027EF25F08251680AD8B4A8EF0EF0825100
:101C8000630AD8B464EF29F08251690AD8B4E5EF49
:101C900020F082517A0AD8B4F8EF21F08251490A33
:101CA000D8B484EF20F08251500AD8B4A2EF1FF0CC
:101CB0008251700AD8B4E5EF1FF08251540AD8B4AB
:101CC00010EF20F08251740AD8B456EF20F0825100
:101CD000410AD8B4ADEF0FF082514B0AD8B4AAEF45
:101CE0000EF082516D0AD8B41DEF14F082514D0AE6
:101CF000D8B436EF14F08251730AD8B457EF24F0F9
:101D00008251530AD8B4BCEF24F082514C0AD8B4A3
:101D1000C5EF14F08251590AD8B46EEF13F012AE29
:101D200001D0128C9BEF29F0040114EE00F08051D9
:101D30007F0BE12682C4E7FF802B120004010D0E09
:101D4000826F94EC0EF00A0E826F94EC0EF012008B
:101D500099EF29F004014B0E826F94EC0EF0040110
:101D60002C0E826F94EC0EF081B802D036B630D0D3
:101D700003018351430AD8B4EFEF0EF003018351FE
:101D8000630AD8B4F1EF0EF003018351520AD8B4BC
:101D9000F3EF0EF003018351720AD8B4F5EF0EF0A1
:101DA00003018351470AD8B4F7EF0EF003018351C2
:101DB000670AD8B4F9EF0EF003018351540AD8B47E
:101DC000FBEF0EF003018351740AD8B46BEF0FF0F0
:101DD00003018351550AD8B4FDEF0EF083D036804D
:101DE0007BD0369079D0368277D0369275D03684D3
:101DF00073D0369471D036866FD084C330F185C3EA
:101E000031F186C332F187C333F10101296BE6EC6E
:101E100030F05DEC30F000C104F101C105F102C108
:101E200006F103C107F1D9EC30F0200EF86EF76A25
:101E3000F66A0900F5CF2CF10900F5CF2DF1090064
:101E4000F5CF2EF10900F5CF2FF10900F5CF30F1D4
:101E50000900F5CF31F10900F5CF32F10900F5CFD6
:101E600033F10101296BE6EC30F05DEC30F083ECEE
:101E70002FF00101006744EF0FF0016744EF0FF00E
:101E8000026744EF0FF0036701D025D004014E0E26
:101E9000826F94EC0EF004016F0E826F94EC0EF0E2
:101EA00004014D0E826F94EC0EF00401610E826FFE
:101EB00094EC0EF00401740E826F94EC0EF00401A9
:101EC000630E826F94EC0EF00401680E826F94EC46
:101ED0000EF099EF29F03696CD0E0C6E36C00BF051
:101EE0004DEC0BF0CD0E64EC0BF0E8CF36F036B0D5
:101EF00006D00401630E826F94EC0EF005D004014D
:101F0000430E826F94EC0EF036B206D00401720ECE
:101F1000826F94EC0EF005D00401520E826F94ECA7
:101F20000EF036B406D00401670E826F94EC0EF00A
:101F300005D00401470E826F94EC0EF036B606D041
:101F40000401740E826F94EC0EF005D00401540E5F
:101F5000826F94EC0EF099EF29F00401410E826F2C
:101F600094EC0EF003018351310AD8B48EEF12F0D5
:101F700003018351320AD8B4BEEF11F0030183513B
:101F8000330AD8B447EF11F003018351340AD8B4AF
:101F900037EF10F003018351350AD8B4D7EF0FF0B3
:101FA00004013F0E826F94EC0EF099EF29F00301CB
:101FB0008451300AD8B4FDEF0FF003018451310A87
:101FC000D8B400EF10F003018451650AD8B4F1EFE2
:101FD0000FF003018451640AD8B4F4EF0FF001EF5D
:101FE00010F03790F5EF0FF03780FB0E0C6E37C016
:101FF0000BF04DEC0BF001EF10F08B9001EF10F0B7
:102000008B800401350E826F94EC0EF004012C0ECF
:10201000826F94EC0EF08BB015EF10F00401300ECF
:10202000826F94EC0EF01AEF10F00401310E826F03
:1020300094EC0EF004012C0E826F94EC0EF0FB0E6B
:1020400064EC0BF0E8CF37F037A02EEF10F004016E
:10205000640E826F94EC0EF033EF10F00401650E05
:10206000826F94EC0EF035EF10F099EF29F0CC0E62
:1020700064EC0BF0E8CF0BF004012C0E826F94ECB3
:102080000EF003018451310AD8B45BEF10F0030164
:102090008451300AD8B45DEF10F0030184514D0A29
:1020A000D8B467EF10F003018451540AD8B46EEF2E
:1020B00010F085EF10F08A8401D08A940BAE04D022
:1020C0000BAC02D00BBA21D0E00E0B1218D01F0EB1
:1020D0000B168539E844E00B0B1211D0E00E0B16FD
:1020E000D9EC30F085C332F186C333F10101296B9D
:1020F000E6EC30F05DEC30F000511F0B0B12CC0E13
:102100000C6E0BC00BF04DEC0BF00401340E826F23
:1021100094EC0EF004012C0E826F94EC0EF0CC0EB9
:1021200064EC0BF0E8CF1DF08AB406D00401300E49
:10213000826F94EC0EF005D00401310E826F94ECA6
:102140000EF004012C0E826F94EC0EF01D38E84066
:10215000070BE8CF82F40401300E822794EC0EF0D6
:1021600004012C0E826F94EC0EF098EC30F01D50B0
:102170001F0BE8CF00F121EC30F032C182F40401F2
:10218000300E822794EC0EF033C182F40401300E3D
:10219000822794EC0EF004012C0E826F94EC0EF06A
:1021A00098EC30F030C000F100AF0BD0FF0E016FA3
:1021B000FF0E026FFF0E036F04012D0E826F94EC71
:1021C0000EF021EC30F031C182F40401300E822790
:1021D00094EC0EF032C182F40401300E822794ECAC
:1021E0000EF033C182F40401300E822794EC0EF01D
:1021F00004012C0E826F94EC0EF098EC30F02FC09E
:1022000000F121EC30F031C182F40401300E82275C
:1022100094EC0EF032C182F40401300E822794EC6B
:102220000EF033C182F40401300E822794EC0EF0DC
:1022300004012C0E826F94EC0EF098EC30F031C05B
:1022400000F100AF0BD0FF0E016FFF0E026FFF0E0B
:10225000036F04012D0E826F94EC0EF021EC30F030
:1022600031C182F40401300E822794EC0EF032C1A9
:1022700082F40401300E822794EC0EF033C182F414
:102280000401300E822794EC0EF099EF29F0CB0E6A
:1022900064EC0BF0E8CF0BF004012C0E826F94EC91
:1022A0000EF003018451450AD8B46BEF11F003011D
:1022B0008451440AD8B46EEF11F003018451300AFE
:1022C000D8B471EF11F003018451310AD8B475EF1D
:1022D00011F080EF11F00B9E7AEF11F00B8E7AEF78
:1022E00011F0FC0E0B167AEF11F0FC0E0B160B80A2
:1022F0007AEF11F0CB0E0C6E0BC00BF04DEC0BF027
:102300000401330E826F94EC0EF004012C0E826FE8
:1023100094EC0EF0CB0E64EC0BF0E8CF1CF01CBE7E
:1023200099EF11F00401450E826F94EC0EF09EEFD0
:1023300011F00401440E826F94EC0EF004012C0E97
:10234000826F94EC0EF00401300E826F94EC0EF06C
:1023500004012C0E826F94EC0EF01CB0B7EF11F05C
:102360000401300E826F94EC0EF0BCEF11F004010A
:10237000310E826F94EC0EF099EF29F0CA0E64ECE6
:102380000BF0E8CF0BF004012C0E826F94EC0EF0F2
:1023900003018451450AD8B4FAEF11F003018451C6
:1023A000440AD8B4FDEF11F0030184514D0AD8B4AA
:1023B00006EF12F003018451410AD8B400EF12F085
:1023C00003018451460AD8B403EF12F0030184518B
:1023D000560AD8B40EEF12F003018451500AD8B453
:1023E00019EF12F003018451520AD8B41CEF12F015
:1023F00025EF12F00B9E1FEF12F00B8E1FEF12F065
:102400000B9C1FEF12F00B8C1FEF12F0FC0E0B1643
:1024100085C3E8FF030B0B121FEF12F0C70E0B165C
:1024200085C3E8FF070BE846E846E8460B121FEFB6
:1024300012F00B841FEF12F00B941FEF12F0CA0E74
:102440000C6E0BC00BF04DEC0BF0CA0E64EC0BF0F5
:10245000E8CF1BF00401320E826F94EC0EF0040101
:102460002C0E826F94EC0EF01BBE3EEF12F00401B6
:10247000450E826F94EC0EF043EF12F00401440E0F
:10248000826F94EC0EF004012C0E826F94EC0EF02F
:102490001BC0E8FF030BE8CF82F40401300E822753
:1024A00094EC0EF004012C0E826F94EC0EF01BBC29
:1024B00061EF12F00401410E826F94EC0EF066EFB2
:1024C00012F00401460E826F94EC0EF004012C0E03
:1024D000826F94EC0EF01BC0E8FF380BE842E84234
:1024E000E842E8CF82F40401300E822794EC0EF02B
:1024F00004012C0E826F94EC0EF01BB487EF12F0E7
:102500000401520E826F94EC0EF08CEF12F0040175
:10251000500E826F94EC0EF099EF29F0C90E64EC26
:102520000BF0E8CF0BF004012C0E826F94EC0EF050
:1025300003018451450AD8B4ACEF12F00301845171
:10254000440AD8B4AFEF12F0030184514D0AD8B455
:10255000B2EF12F0C0EF12F00B9EBAEF12F00B8E3A
:10256000BAEF12F0F80E0B1685C3E8FF070B0B123B
:10257000BAEF12F0C90E0C6E0BC00BF04DEC0BF065
:102580000401310E826F94EC0EF004012C0E826F68
:1025900094EC0EF0C90E64EC0BF0E8CF1AF01ABE02
:1025A00006D00401450E826F94EC0EF005D00401B4
:1025B000440E826F94EC0EF004012C0E826F94ECAA
:1025C0000EF01AC0E8FF070BE8CF82F40401300ECA
:1025D000822794EC0EF004012C0E826F94EC0EF026
:1025E000078098EC30F02BC0E8FF003B004300432D
:1025F000030B21EC30F033C182F40401300E82274A
:1026000094EC0EF004012C0E826F94EC0EF098EC1A
:1026100030F02BC001F1019F019D2CC000F10101A0
:1026200021EC30F02FC182F40401300E822794ECAB
:102630000EF030C182F40401300E822794EC0EF0CB
:1026400031C182F40401300E822794EC0EF032C1C5
:1026500082F40401300E822794EC0EF033C182F430
:102660000401300E822794EC0EF004012C0E826FD0
:1026700094EC0EF098EC30F02DC001F12EC000F17A
:10268000D89001330033D89001330033010121EC9D
:1026900030F02FC182F40401300E822794EC0EF04A
:1026A00030C182F40401300E822794EC0EF031C167
:1026B00082F40401300E822794EC0EF032C182F4D1
:1026C0000401300E822794EC0EF033C182F4040131
:1026D000300E822794EC0EF099EF29F0FC0E64EC9A
:1026E0000BF0E8CF0BF003018351520AD8B4A5EFE9
:1026F00013F003018351720AD8B4A8EF13F0030159
:102700008351500AD8B4ABEF13F003018351700A20
:10271000D8B4AEEF13F003018351550AD8B4B1EF2A
:1027200013F003018351750AD8B4B4EF13F0030119
:102730008351430AD8B4BDEF13F003018351630AF8
:10274000D8B4C0EF13F0C9EF13F00B90C3EF13F040
:102750000B80C3EF13F00B92C3EF13F00B82C3EFA8
:1027600013F00B94C3EF13F00B84C3EF13F00B962D
:10277000C3EF13F00B86C3EF13F00B98C3EF13F006
:102780000B88C3EF13F0FC0E0C6E0BC00BF04DEC7E
:102790000BF00401590E826F94EC0EF0119011921F
:1027A00011941198FC0E64EC0BF0E8CF0BF00BA029
:1027B00011800BA211820BA411840BA8118811A007
:1027C000E9EF13F00401520E826F94EC0EF0EEEF7D
:1027D00013F00401720E826F94EC0EF011A8F8EF62
:1027E00013F00401430E826F94EC0EF0FDEF13F032
:1027F0000401630E826F94EC0EF011A207EF14F047
:102800000401500E826F94EC0EF00CEF14F00401F2
:10281000700E826F94EC0EF011A416EF14F0040108
:10282000550E826F94EC0EF01BEF14F00401750E40
:10283000826F94EC0EF099EF29F004016D0E826F17
:1028400094EC0EF003018351300AD8B475EF14F004
:1028500003018351310AD8B488EF14F00301835186
:10286000320AD8B49BEF14F09BEF29F004014D0E0F
:10287000826F94EC0EF0D9EC30F084C331F185C353
:1028800032F186C333F10101296BE6EC30F05DECE7
:1028900030F003018351300AD8B45DEF14F0030126
:1028A0008351310AD8B465EF14F003018351320A21
:1028B000D8B46DEF14F09BEF29F0FD0E0C6E00C143
:1028C0000BF04DEC0BF075EF14F0FE0E0C6E00C12A
:1028D0000BF04DEC0BF088EF14F0FF0E0C6E00C106
:1028E0000BF04DEC0BF09BEF14F00401300E826FF7
:1028F00094EC0EF004012C0E826F94EC0EF098EC28
:1029000030F0FD0E64EC0BF0E8CF00F1ACEF14F00A
:102910000401310E826F94EC0EF004012C0E826FD4
:1029200094EC0EF098EC30F0FE0E64EC0BF0E8CF77
:1029300000F1ACEF14F00401320E826F94EC0EF053
:1029400098EC30F004012C0E826F94EC0EF0FF0E28
:1029500064EC0BF0E8CF00F121EC30F031C182F4EF
:102960000401300E822794EC0EF032C182F404018F
:10297000300E822794EC0EF033C182F40401300E45
:10298000822794EC0EF099EF29F003018351300A6D
:10299000D8B419EF1AF003018351310AD8B446EFC5
:1029A0001BF003018351320AD8B4B4EF1BF00301CA
:1029B0008351330AD8B4C4EF1BF003018351340AA6
:1029C000D8B41FEF1CF003018351350AD8B4F3EFDC
:1029D0001DF003018351360AD8B421EF1EF0030124
:1029E0008351370AD8B4F1EF17F003018351380A45
:1029F000D8B48FEF18F003018351440AD8B41DEF07
:102A000016F003018351640AD8B43DEF16F00301B8
:102A10008351460AD8B4F8EF1CF0030183514D0AE4
:102A2000D8B46AEF16F0030183516D0AD8B484EF6D
:102A300016F0030183515A0AD8B4C0EF1AF003010B
:102A40008351490AD8B421EF1FF003018351500A82
:102A5000D8B453EF1EF003018351540AD8B4CCEF1D
:102A60001EF003018351630AD8B4A4EF16F00301EA
:102A70008351430AD8B49CEF17F003018351730AC2
:102A8000D8B4A2EF16F003018351610AD8B46AEFFB
:102A900015F003018351650AD8B469EF1AF00301F8
:102AA0008351450AD8B477EF1AF003018351620AC3
:102AB000D8B485EF1AF003018351420AD8B493EFDA
:102AC0001AF003018351760AD8B4A1EF1AF0D8A402
:102AD0009BEF29F004014C0E826F94EC0EF0040180
:102AE000610E826F94EC0EF0E1EC31F004012C0EDB
:102AF000826F94EC0EF098EC30F0AFC500F101015C
:102B000021EC30F031C182F40401300E822794ECC4
:102B10000EF032C182F40401300E822794EC0EF0E4
:102B200033C182F40401300E822794EC0EF00401CC
:102B30002C0E826F94EC0EF098EC30F0B0C500F1E2
:102B4000010121EC30F031C182F40401300E822702
:102B500094EC0EF032C182F40401300E822794EC22
:102B60000EF033C182F40401300E822794EC0EF093
:102B700004012C0E826F94EC0EF098EC30F0B1C58D
:102B800000F1010121EC30F031C182F40401300E7A
:102B9000822794EC0EF032C182F40401300E8227B9
:102BA00094EC0EF033C182F40401300E822794ECD1
:102BB0000EF004012C0E826F94EC0EF098EC30F0C5
:102BC000B2C500F1010121EC30F031C182F4040101
:102BD000300E822794EC0EF032C182F40401300EE4
:102BE000822794EC0EF033C182F40401300E822768
:102BF00094EC0EF004012C0E826F94EC0EF098EC25
:102C000030F0B6C500F1010121EC30F031C182F4A1
:102C10000401300E822794EC0EF032C182F40401DC
:102C2000300E822794EC0EF033C182F40401300E92
:102C3000822794EC0EF04FEF1EF003018451300A0E
:102C4000D8B429EF16F003018451310AD8B42DEF1E
:102C500016F0159215962EEF16F01582C70E64EC3D
:102C60000BF0E8CF00F10101008115A20091C70E21
:102C70000C6E00C10BF04DEC0BF0C70E64EC0BF0CA
:102C8000E8CF00F1010100B149EF16F015924AEFCB
:102C900016F0158204014C0E826F94EC0EF00401C4
:102CA000640E826F94EC0EF004012C0E826F94EC93
:102CB0000EF015B263EF16F00401300E826F94EC43
:102CC0000EF068EF16F00401310E826F94EC0EF0F6
:102CD00099EF29F0D9EC30F084C333F1E6EC30F011
:102CE0005DEC30F0200E0C6E00C10BF04DEC0BF0E3
:102CF00000C12FF505012F51000A06E005012F51F3
:102D0000010A02E07BEC32F004014C0E826F94EC7D
:102D10000EF004014D0E826F94EC0EF004012C0EA7
:102D2000826F94EC0EF098EC30F02FC500F121EC9E
:102D300030F033C182F40401300E822794EC0EF09F
:102D40004FEF1EF05DEF38F004014C0E826F94ECF3
:102D50000EF00401630E826F94EC0EF039EC31F04A
:102D600004012C0E826F94EC0EF0B9EC16F04FEFCC
:102D70001EF098EC30F0B5C500F10101003B0F0EDC
:102D8000001721EC30F033C182F40401300E8227A9
:102D900094EC0EF0B5C500F101010F0E0101001712
:102DA00021EC30F033C182F40401300E822794EC20
:102DB0000EF004012D0E826F94EC0EF0B4C500F1FC
:102DC0000101003B0F0E001721EC30F033C182F4FB
:102DD0000401300E822794EC0EF0B4C500F101011D
:102DE0000F0E0101001721EC30F033C182F4040111
:102DF000300E822794EC0EF004012D0E826F94ECBD
:102E00000EF0B3C500F10101003B0F0E001721ECDD
:102E100030F033C182F40401300E822794EC0EF0BE
:102E2000B3C500F101010F0E0101001721EC30F0D4
:102E300033C182F40401300E822794EC0EF00401B9
:102E4000200E826F94EC0EF0B2C500F10F0E01015E
:102E5000001721EC30F033C182F40401300E8227D8
:102E600094EC0EF00401200E826F94EC0EF0B1C5CC
:102E700000F101010101003B0F0E001721EC30F0C1
:102E800033C182F40401300E822794EC0EF0B1C5F8
:102E900000F101010F0E0101001721EC30F033C1E8
:102EA00082F40401300E822794EC0EF004013A0EF5
:102EB000826F94EC0EF0B0C500F10101003B0F0EE3
:102EC000001721EC30F033C182F40401300E822768
:102ED00094EC0EF0B0C500F101010F0E01010017D6
:102EE00021EC30F033C182F40401300E822794ECDF
:102EF0000EF004013A0E826F94EC0EF0AFC500F1B3
:102F00000101003B0F0E001721EC30F033C182F4B9
:102F10000401300E822794EC0EF0AFC500F10101E0
:102F20000F0E001721EC30F033C182F40401300E93
:102F3000822794EC0EF0120084C3E8FF0F0BE83AEE
:102F4000E8CFB5F585C3E8FF0F0B0501B51387C3BF
:102F5000E8FF0F0BE83AE8CFB4F588C3E8FF0F0BA2
:102F60000501B4138AC3E8FF0F0BE83AE8CFB3F5C5
:102F70008BC3E8FF0F0B0501B3138DC3E8FF0F0BE5
:102F8000E8CFB2F58FC3E8FF0F0BE83AE8CFB1F511
:102F900090C3E8FF0F0B0501B11392C3E8FF0F0BBD
:102FA000E83AE8CFB0F593C3E8FF0F0B0501B01383
:102FB00095C3E8FF0F0BE83AE8CFAFF596C3E8FFFB
:102FC0000F0B0501AF1394EC31F004014C0E826F2E
:102FD00094EC0EF00401430E826F94EC0EF0AEEF11
:102FE00016F0078404014C0E826F94EC0EF004017D
:102FF000370E826F94EC0EF004012C0E826F94EC6D
:103000000EF005012E51130A06E005012E51170A94
:103010000DE08CEF18F00101000E006F000E016F43
:10302000100E026F000E036F1FEF18F00101000E6B
:10303000006F000E016F000E026F010E036F21EC96
:1030400030F02AC182F40401300E822794EC0EF095
:103050002BC182F40401300E822794EC0EF02CC1B7
:1030600082F40401300E822794EC0EF02DC182F41C
:103070000401300E822794EC0EF02EC182F404017C
:10308000300E822794EC0EF02FC182F40401300E32
:10309000822794EC0EF030C182F40401300E8227B6
:1030A00094EC0EF031C182F40401300E822794ECCE
:1030B0000EF032C182F40401300E822794EC0EF03F
:1030C00033C182F40401300E822794EC0EF0040127
:1030D0002C0E826F94EC0EF00101100E006F000EAA
:1030E000016F000E026F000E036F21EC30F031C152
:1030F00082F40401300E822794EC0EF032C182F487
:103100000401300E822794EC0EF033C182F40401E6
:10311000300E822794EC0EF007944FEF1EF005015D
:10312000216B226B236B246B04014C0E826F94EC99
:103130000EF00401380E826F94EC0EF004012C0E98
:10314000826F94EC0EF00101100E006F000E016F03
:10315000000E026F000E036F21EC30F02AC182F4E2
:103160000401300E822794EC0EF02BC182F404018E
:10317000300E822794EC0EF02CC182F40401300E44
:10318000822794EC0EF02DC182F40401300E8227C8
:1031900094EC0EF02EC182F40401300E822794ECE0
:1031A0000EF02FC182F40401300E822794EC0EF051
:1031B00030C182F40401300E822794EC0EF031C14C
:1031C00082F40401300E822794EC0EF032C182F4B6
:1031D0000401300E822794EC0EF033C182F4040116
:1031E000300E822794EC0EF004012C0E826F94ECCA
:1031F0000EF025C500F126C501F127C502F128C54D
:1032000003F10101100E046F000E056F000E066F32
:10321000000E076FB4EC2FF000C133F501C134F597
:1032200002C135F503C136F521EC30F02AC182F434
:103230000401300E822794EC0EF02BC182F40401BD
:10324000300E822794EC0EF02CC182F40401300E73
:10325000822794EC0EF02DC182F40401300E8227F7
:1032600094EC0EF02EC182F40401300E822794EC0F
:103270000EF02FC182F40401300E822794EC0EF080
:1032800030C182F40401300E822794EC0EF031C17B
:1032900082F40401300E822794EC0EF032C182F4E5
:1032A0000401300E822794EC0EF033C182F4040145
:1032B000300E822794EC0EF09EEC0EF00501336781
:1032C00069EF19F0346769EF19F0356769EF19F0A4
:1032D000366702D008EF1AF0129E129C21C500F149
:1032E00022C501F123C502F124C503F1899A400EDC
:1032F000C76E200EC66E9E96C69E0B0EC96EFF0E42
:103300009EB602D0E82EFCD79E96C69E02C1C9FF8B
:10331000FF0E9EB602D0E82EFCD79E96C69E01C137
:10332000C9FFFF0E9EB602D0E82EFCD79E96C69E21
:1033300000C1C9FFFF0E9EB602D0E82EFCD79E96B4
:10334000C69EC952FF0E9EB602D0E82EFCD70501DC
:10335000100E326F040114EE00F080517F0BE12655
:103360009E96C69EC952FF0E9EB602D0E82EFCD78E
:10337000C9CFE7FF0401802B0501322FAAEF19F016
:10338000898A33C500F134C501F135C502F136C56E
:1033900003F10101010E046F000E056F000E066FB0
:1033A000000E076F83EC2FF000C133F501C134F537
:1033B00002C135F503C136F505013367E7EF19F0B2
:1033C0003467E7EF19F03567E7EF19F0366702D099
:1033D00008EF1AF021C500F122C501F123C502F161
:1033E00024C503F10101100E046F000E056F000EDD
:1033F000066F000E076F88EC2FF000C121F501C1A8
:1034000022F502C123F503C124F5128E9BEF29F0AA
:103410000401450E826F94EC0EF004014F0E826F92
:1034200094EC0EF00401460E826F94EC0EF04FEF18
:103430001EF00784B7EC37F098EC30F02DC500F1A2
:1034400021EC30F004014C0E826F94EC0EF004017C
:10345000300E826F94EC0EF004012C0E826F94EC0F
:103460000EF031C182F40401300E822794EC0EF08C
:1034700032C182F40401300E822794EC0EF033C185
:1034800082F40401300E822794EC0EF004012C0E1D
:10349000826F94EC0EF098EC30F02EC500F121EC28
:1034A00030F031C182F40401300E822794EC0EF02A
:1034B00032C182F40401300E822794EC0EF033C145
:1034C00082F40401300E822794EC0EF007944FEF43
:1034D0001EF004014C0E826F94EC0EF00401650E98
:1034E000826F94EC0EF057EC33F04FEF1EF00401B6
:1034F0004C0E826F94EC0EF00401450E826F94EC3A
:103500000EF06EEC33F04FEF1EF004014C0E826FA4
:1035100094EC0EF00401620E826F94EC0EF09CECC1
:1035200033F04FEF1EF004014C0E826F94EC0EF05E
:103530000401420E826F94EC0EF085EC33F04FEFF5
:103540001EF004014C0E826F94EC0EF00401760E16
:10355000826F94EC0EF004012C0E826F94EC0EF04E
:1035600010A807D00401310E826F94EC0EF04FEFDB
:103570001EF00401300E826F94EC0EF04FEF1EF03F
:1035800004014C0E826F94EC0EF004015A0E826F0F
:1035900094EC0EF004012C0E826F94EC0EF0B7EC5C
:1035A00037F098EC30F005012E51130A06E00501C2
:1035B0002E51170A0DE0F1EF1AF00101000E006F15
:1035C000000E016F100E026F000E036FF1EF1AF084
:1035D0000101000E006F000E016F000E026F010E60
:1035E000036F0101100E046F000E056F000E066FD1
:1035F000000E076FB4EC2FF021EC30F02AC182F4FA
:103600000401300E822794EC0EF02BC182F40401E9
:10361000300E822794EC0EF02CC182F40401300E9F
:10362000822794EC0EF02DC182F40401300E822723
:1036300094EC0EF02EC182F40401300E822794EC3B
:103640000EF02FC182F40401300E822794EC0EF0AC
:1036500030C182F40401300E822794EC0EF031C1A7
:1036600082F40401300E822794EC0EF032C182F411
:103670000401300E822794EC0EF033C182F4040171
:10368000300E822794EC0EF04FEF1EF007840401F9
:103690004C0E826F94EC0EF00401310E826F94ECAC
:1036A0000EF004012C0E826F94EC0EF025C500F193
:1036B00026C501F127C502F128C503F10101100E4D
:1036C000046F000E056F000E066F000E076FB4EC5E
:1036D0002FF021EC30F02AC182F40401300E822751
:1036E00094EC0EF02BC182F40401300E822794EC8E
:1036F0000EF02CC182F40401300E822794EC0EF0FF
:103700002DC182F40401300E822794EC0EF02EC1FC
:1037100082F40401300E822794EC0EF02FC182F463
:103720000401300E822794EC0EF030C182F40401C3
:10373000300E822794EC0EF031C182F40401300E79
:10374000822794EC0EF032C182F40401300E8227FD
:1037500094EC0EF033C182F40401300E822794EC15
:103760000EF007944FEF1EF0078404014C0E826F99
:1037700094EC0EF00401320E826F94EC0EF08BECA0
:1037800035F007944FEF1EF0078437B0CAEF1BF0F7
:10379000DDEF1BF0010E166E04014C0E826F94ECEF
:1037A0000EF00401330E826F94EC0EF0E8EC35F06D
:1037B000000E166E079451EF1BF0020E166EE8EC29
:1037C00035F08B800501010E306F3C0E316F010129
:1037D0005E6B5F6B606B616B626B636B646B656B85
:1037E000666B676B686B696B536B546BCF6ACE6AA1
:1037F0000F9A0F9C0F9E030E166E04014C0E826FE3
:1038000094EC0EF00401330E826F94EC0EF0040180
:103810002C0E826F94EC0EF004012D0E826F94EC4E
:103820000EF00401310E826F94EC0EF099EF29F046
:10383000E8EC35F0000E166E8B909BEF29F00784B4
:1038400004014C0E826F94EC0EF00401340E826F72
:1038500094EC0EF004012C0E826F94EC0EF0D9EC77
:1038600030F084C32AF185C32BF186C32CF187C3C2
:103870002DF188C32EF189C32FF18AC330F18BC398
:1038800031F18CC332F18DC333F10101296BE6ECC8
:1038900030F05DEC30F0100E046F000E056F000E7E
:1038A000066F000E076F94EC2FF000C121F501C1E7
:1038B00022F502C123F503C124F56AEC37F038C5BF
:1038C000AFF539C5B0F53AC5B1F53BC5B2F53CC564
:1038D000B3F53DC5B4F53EC5B5F5B9EC16F0040138
:1038E0002C0E826F94EC0EF03FC500F140C501F143
:1038F00041C502F142C503F10101000E046F000E43
:10390000056F010E066F000E076FB4EC2FF021EC6F
:1039100030F029678EEF1CF093EF1CF004012D0EA0
:10392000826F94EC0EF030C182F40401300E8227D5
:1039300094EC0EF031C182F40401300E822794EC35
:103940000EF004012E0E826F94EC0EF032C182F460
:103950000401300E822794EC0EF033C182F404018E
:10396000300E822794EC0EF004012C0E826F94EC42
:103970000EF098EC30F043C500F144C501F1C5EC00
:103980002AF004012C0E826F94EC0EF098EC30F0CB
:1039900045C500F121EC30F031C182F40401300E54
:1039A000822794EC0EF032C182F40401300E82279B
:1039B00094EC0EF033C182F40401300E822794ECB3
:1039C0000EF004012C0E826F94EC0EF037C5E8FF68
:1039D000E8B806D00401300E826F94EC0EF005D0EA
:1039E0000401310E826F94EC0EF007944FEF1EF03D
:1039F000D9EC30F085C32AF186C32BF187C32CF1B3
:103A000088C32DF189C32EF18AC32FF18BC330F106
:103A10008CC331F18DC332F18EC333F10101296BB7
:103A2000E6EC30F05DEC30F00101010E046F000EA9
:103A3000056F000E066F000E076F83EC2FF0100E5F
:103A4000046F000E056F000E066F000E076F94ECFA
:103A50002FF000C129F501C12AF502C12BF503C1E0
:103A60002CF512EC35F004014C0E826F94EC0EF044
:103A70000401460E826F94EC0EF004012C0E826F4E
:103A800094EC0EF025C500F126C501F127C502F121
:103A900028C503F10101100E046F000E056F000E22
:103AA000066F000E076FB4EC2FF021EC30F02AC146
:103AB00082F40401300E822794EC0EF02BC182F4C4
:103AC0000401300E822794EC0EF02CC182F4040124
:103AD000300E822794EC0EF02DC182F40401300EDA
:103AE000822794EC0EF02EC182F40401300E82275E
:103AF00094EC0EF02FC182F40401300E822794EC76
:103B00000EF030C182F40401300E822794EC0EF0E6
:103B100031C182F40401300E822794EC0EF032C1E0
:103B200082F40401300E822794EC0EF033C182F44B
:103B30000401300E822794EC0EF04FEF1EF037B0E8
:103B4000A4EF1DF0020E166EE8EC35F000011650E1
:103B5000020AD8B4C2EF1DF005012F51010AD8B4F2
:103B6000B8EF1DF015B2BDEF1DF081BABDEF1DF02D
:103B7000000E166E15849BEF29F0050E166E158447
:103B80005DEF38F08B8001015E6B5F6B606B616B8A
:103B9000626B636B646B656B666B676B686B696BA1
:103BA000536B546BCF6ACE6A0F9A0F9C0F9E030E15
:103BB000166E9BEF29F0E8EC35F005012F51010A54
:103BC000D8B4E9EF1DF015B2EEEF1DF081BAEEEFBB
:103BD0001DF0000E166E15849BEF29F0050E166E73
:103BE00015845DEF38F004014C0E826F94EC0EF0FA
:103BF0000401350E826F94EC0EF004012C0E826FDE
:103C000094EC0EF098EC30F00784B9C500F10794FD
:103C100021EC30F031C182F40401300E822794ECA3
:103C20000EF032C182F40401300E822794EC0EF0C3
:103C300033C182F40401300E822794EC0EF04FEF72
:103C40001EF0ABEC35F098EC30F037C500F121EC0C
:103C500030F004014C0E826F94EC0EF00401360E2D
:103C6000826F94EC0EF004012C0E826F94EC0EF037
:103C700031C182F40401300E822794EC0EF032C17F
:103C800082F40401300E822794EC0EF033C182F4EA
:103C90000401300E822794EC0EF04FEF1EF09EECE4
:103CA0000EF09BEF29F004014C0E826F94EC0EF0A5
:103CB0000401500E826F94EC0EF004012C0E826F02
:103CC00094EC0EF085C32AF186C32BF187C32CF147
:103CD00088C32DF189C32EF18AC32FF18BC330F134
:103CE0008CC331F18DC332F18EC333F10101E6ECA7
:103CF00030F05DEC30F003018451530A0DE0030114
:103D000084514D0A38E00401780E826F94EC0EF075
:103D10009EEC0EF09BEF29F00401530E826F94ECA1
:103D20000EF0250E0C6E00C10BF04DEC0BF0260EC4
:103D30000C6E01C10BF04DEC0BF0270E0C6E02C1A6
:103D40000BF04DEC0BF0280E0C6E03C10BF04DEC9C
:103D50000BF000C157F501C158F502C159F503C177
:103D60005AF500C15BF501C15CF502C15DF503C107
:103D70005EF530EF1FF004014D0E826F94EC0EF0F3
:103D8000290E0C6E00C10BF04DEC0BF000C15FF57D
:103D900000C160F530EF1FF004014C0E826F94EC0F
:103DA0000EF00401540E826F94EC0EF004012C0E00
:103DB000826F94EC0EF084C32AF185C32BF186C385
:103DC0002CF187C32DF188C32EF189C32FF18AC34B
:103DD00030F18BC331F18DC332F18EC333F1010168
:103DE000E6EC30F05DEC30F00101000E046F000EE7
:103DF000056F010E066F000E076F94EC2FF0210E79
:103E00000C6E00C10BF04DEC0BF0220E0C6E01C1DC
:103E10000BF04DEC0BF0230E0C6E02C10BF04DECD1
:103E20000BF0240E0C6E03C10BF04DEC0BF000C137
:103E300061F501C162F502C163F503C164F530EFBC
:103E40001FF004014C0E826F94EC0EF00401490E39
:103E5000826F94EC0EF004012C0E826F94EC0EF045
:103E6000250E64EC0BF0E8CF00F1260E64EC0BF0AD
:103E7000E8CF01F1270E64EC0BF0E8CF02F1280E39
:103E800064EC0BF0E8CF03F121EC30F0E4EC2DF022
:103E90000401730E826F94EC0EF004012C0E826FFD
:103EA00094EC0EF098EC30F0290E64EC0BF0E8CFB7
:103EB00000F121EC30F0E4EC2DF004016D0E826F86
:103EC00094EC0EF004012C0E826F94EC0EF05BC5A6
:103ED00000F15CC501F15DC502F15EC503F121ECA5
:103EE00030F0E4EC2DF00401730E826F94EC0EF0D0
:103EF00004012C0E826F94EC0EF098EC30F060C54B
:103F000000F121EC30F0E4EC2DF004016D0E826F35
:103F100094EC0EF004012C0E826F94EC0EF061C54F
:103F200000F162C501F163C502F164C503F1B6ECAD
:103F300029F004012C0E826F94EC0EF09EEC0EF032
:103F40009BEF29F083C32AF184C32BF185C32CF1A5
:103F500086C32DF187C32EF188C32FF189C330F1B9
:103F60008AC331F18BC332F18CC333F10101E6EC2A
:103F700030F05DEC30F0160E0C6E00C10BF04DEC25
:103F80000BF0170E0C6E01C10BF04DEC0BF0180E80
:103F90000C6E02C10BF04DEC0BF0190E0C6E03C150
:103FA0000BF04DEC0BF000C18EF101C18FF102C19D
:103FB00090F103C191F100C192F101C193F102C1ED
:103FC00094F103C195F184EF20F083C32AF184C3F7
:103FD0002BF185C32CF186C32DF187C32EF188C345
:103FE0002FF189C330F18AC331F18BC332F18CC315
:103FF00033F10101E6EC30F05DEC30F000C18EF100
:1040000001C18FF102C190F103C191F100C192F1A0
:1040100001C193F102C194F103C195F184EF20F045
:1040200083C32AF184C32BF185C32CF186C32DF100
:1040300087C32EF188C32FF189C330F18AC331F1D0
:104040008CC332F18DC333F10101E6EC30F05DEC4D
:1040500030F00101000E046F000E056F010E066FB7
:10406000000E076F94EC2FF01A0E0C6E00C10BF0CF
:104070004DEC0BF01B0E0C6E01C10BF04DEC0BF078
:104080001C0E0C6E02C10BF04DEC0BF01D0E0C6EF5
:1040900003C10BF04DEC0BF000C196F101C197F19B
:1040A00002C198F103C199F184EF20F083C32AF192
:1040B00084C32BF185C32CF186C32DF187C32EF168
:1040C00088C32FF189C330F18AC331F18CC332F137
:1040D0008DC333F10101E6EC30F05DEC30F001010D
:1040E000000E046F000E056F010E066F000E076FC5
:1040F00094EC2FF000C196F101C197F102C198F143
:1041000003C199F184EF20F0160E64EC0BF0E8CFB8
:1041100000F1170E64EC0BF0E8CF01F1180E64EC1F
:104120000BF0E8CF02F1190E64EC0BF0E8CF03F1CD
:1041300021EC30F0E4EC2DF00401730E826F94EC6E
:104140000EF004012C0E826F94EC0EF08EC100F183
:104150008FC101F190C102F191C103F121EC30F066
:10416000E4EC2DF00401730E826F94EC0EF0040168
:104170002C0E826F94EC0EF01A0E64EC0BF0E8CF6C
:1041800000F11B0E64EC0BF0E8CF01F11C0E64ECA7
:104190000BF0E8CF02F11D0E64EC0BF0E8CF03F159
:1041A000B6EC29F004012C0E826F94EC0EF096C14F
:1041B00000F197C101F198C102F199C103F1B6EC88
:1041C00029F09EEC0EF09BEF29F00401690E826F3E
:1041D00094EC0EF004012C0E826F94EC0EF00101B1
:1041E000040E006F000E016F000E026F000E036FD1
:1041F00021EC30F02CC182F40401300E822794ECC3
:104200000EF02DC182F40401300E822794EC0EF0E2
:104210002EC182F40401300E822794EC0EF02FC1DF
:1042200082F40401300E822794EC0EF030C182F447
:104230000401300E822794EC0EF031C182F40401A7
:10424000300E822794EC0EF032C182F40401300E5D
:10425000822794EC0EF033C182F40401300E8227E1
:1042600094EC0EF004012C0E826F94EC0EF0010120
:10427000060E006F000E016F000E026F000E036F3E
:1042800021EC30F02CC182F40401300E822794EC32
:104290000EF02DC182F40401300E822794EC0EF052
:1042A0002EC182F40401300E822794EC0EF02FC14F
:1042B00082F40401300E822794EC0EF030C182F4B7
:1042C0000401300E822794EC0EF031C182F4040117
:1042D000300E822794EC0EF032C182F40401300ECD
:1042E000822794EC0EF033C182F40401300E822751
:1042F00094EC0EF004012C0E826F94EC0EF0010190
:10430000480E006F000E016F000E026F000E036F6B
:1043100021EC30F02CC182F40401300E822794ECA1
:104320000EF02DC182F40401300E822794EC0EF0C1
:104330002EC182F40401300E822794EC0EF02FC1BE
:1043400082F40401300E822794EC0EF030C182F426
:104350000401300E822794EC0EF031C182F4040186
:10436000300E822794EC0EF032C182F40401300E3C
:10437000822794EC0EF033C182F40401300E8227C0
:1043800094EC0EF004012C0E826F94EC0EF0200ED3
:10439000F86EF76AF66A04010900F5CF82F494EC2E
:1043A0000EF00900F5CF82F494EC0EF00900F5CF81
:1043B00082F494EC0EF00900F5CF82F494EC0EF048
:1043C0000900F5CF82F494EC0EF00900F5CF82F4E9
:1043D00094EC0EF00900F5CF82F494EC0EF0090095
:1043E000F5CF82F494EC0EF09EEC0EF09BEF29F0EA
:1043F0008351630AD8A499EF29F08451610AD8A4A3
:1044000099EF29F085516C0AD8A499EF29F08651CB
:10441000410A3FE08651440A1BE08651420AD8B463
:104420005CEF22F08651350AD8B425EF2BF0865187
:10443000360AD8B47AEF2BF08651370AD8B4E3EFB6
:104440002BF08651380AD8B441EF2CF099EF29F0BF
:104450000798079A04017A0E826F94EC0EF004011B
:10446000780E826F94EC0EF00401640E826F94EC6F
:104470000EF00401550E826F94EC0EF045EF22F021
:1044800004014C0E826F94EC0EF09EEC0EF09BEF4C
:1044900029F00788079A04017A0E826F94EC0EF0D7
:1044A0000401410E826F94EC0EF00401610E826FE4
:1044B00094EC0EF039EF22F00798078A04017A0E87
:1044C000826F94EC0EF00401420E826F94EC0EF0B9
:1044D0000401610E826F94EC0EF039EF22F00101BD
:1044E00066677AEF22F067677AEF22F068677AEF03
:1044F00022F0696716D001014F6786EF22F05067FE
:1045000086EF22F0516786EF22F052670AD0010150
:10451000000E006F000E016F000E026F000E036FA1
:10452000120011B80AD00101620E046F010E056F6E
:10453000000E066F000E076F09D00101A70E046F71
:10454000020E056F000E066F000E076F66C100F1C8
:1045500067C101F168C102F169C103F183EC2FF079
:1045600003BF23EF23F0119A119C0101000E046F89
:10457000A80E056F550E066F020E076F66C100F19B
:1045800067C101F168C102F169C103F166C18AF135
:1045900067C18BF168C18CF169C18DF183EC2FF09B
:1045A00003BF0BD00101000E8A6FA80E8B6F550E52
:1045B0008C6F020E8D6F118A119C0E0E64EC0BF045
:1045C000E8CF18F10F0E64EC0BF0E8CF19F1100EE4
:1045D00064EC0BF0E8CF1AF1110E64EC0BF0E8CFAD
:1045E0001BF1CCEC2EF08AC104F18BC105F18CC11A
:1045F00006F18DC107F183EC2FF0078290EC2EF0CD
:10460000CCEC2EF0079290EC2EF08AC100F18BC119
:1046100001F18CC102F18DC103F1079290EC2EF0F3
:10462000CC0E046FE00E056F870E066F050E076F48
:1046300083EC2FF000C118F101C119F102C11AF188
:1046400003C11BF140D013AA28EF23F0138E139A55
:10465000119C119A0101800E006F1A0E016F060E57
:10466000026F000E036F4FC104F150C105F151C13B
:1046700006F152C107F183EC2FF003AF05D098EC9F
:1046800030F0118C119A12000E0E64EC0BF0E8CF92
:1046900018F10F0E64EC0BF0E8CF19F1100E64EC7A
:1046A0000BF0E8CF1AF1110E64EC0BF0E8CF1BF120
:1046B0004FC100F150C101F151C102F152C103F1EA
:1046C000078290EC2EF018C100F119C101F11AC156
:1046D00002F11BC103F112000784BAC166F1BBC12C
:1046E00067F1BCC168F1BDC169F14BC14FF14CC16B
:1046F00050F14DC151F14EC152F157C159F158C15C
:104700005AF10794010166678DEF23F067678DEF1B
:1047100023F068678DEF23F0696716D001014F67BA
:1047200099EF23F0506799EF23F0516799EF23F049
:1047300052670AD00101000E006F000E016F000EDB
:10474000026F000E036F120011B80AD00101620E51
:10475000046F010E056F000E066F000E076F09D083
:104760000101A70E046F020E056F000E066F000E0A
:10477000076F66C100F167C101F168C102F169C14B
:1047800003F183EC2FF003BF25EF24F00101000EAD
:10479000046FA80E056F550E066F020E076F66C1F7
:1047A00000F167C101F168C102F169C103F166C19D
:1047B0008AF167C18BF168C18CF169C18DF183EC1D
:1047C0002FF003BF09D00101000E8A6FA80E8B6F76
:1047D000550E8C6F020E8D6FCCEC2EF000C104F1E3
:1047E00001C105F102C106F103C107F1000E006F1E
:1047F000A00E016F980E026F7B0E036FB4EC2FF0CA
:1048000000C118F101C119F102C11AF103C11BF174
:10481000000E006FA00E016F980E026F7B0E036FEB
:104820008AC104F18BC105F18CC106F18DC107F17C
:10483000B4EC2FF018C104F119C105F11AC106F149
:104840001BC107F183EC2FF012000101A80E006FCD
:10485000610E016F000E026F000E036F4FC104F175
:1048600050C105F151C106F152C107F183EC2FF09F
:1048700003AF0AD00101A80E006F610E016F000E98
:10488000026F000E036F00D0C80E006FAF0E016FF5
:10489000000E026F000E036F4FC104F150C105F10D
:1048A00051C106F152C107F194EC2FF0120004013E
:1048B000730E826F94EC0EF004012C0E826F94EC58
:1048C0000EF0078462C166F163C167F164C168F1EB
:1048D00065C169F14BC14FF14CC150F14DC151F16E
:1048E0004EC152F157C159F158C15AF107947DECAC
:1048F00024F09EEC0EF09BEF29F066C100F167C139
:1049000001F168C102F169C103F1010121EC30F04C
:10491000E4EC2DF00401630E826F94EC0EF00401C0
:104920002C0E826F94EC0EF04FC100F150C101F1DA
:1049300051C102F152C103F1010121EC30F0E4EC6C
:104940002DF00401660E826F94EC0EF004012C0E23
:10495000826F94EC0EF098EC30F059C100F15AC11E
:1049600001F1010121EC30F0E4EC2DF00401740EB2
:10497000826F94EC0EF0120010820401530E826FCD
:1049800094EC0EF004012C0E826F94EC0EF083C3B5
:104990002AF184C32BF185C32CF186C32DF187C383
:1049A0002EF188C32FF189C330F18AC331F18BC353
:1049B00032F18CC333F10101E6EC30F05DEC30F004
:1049C00000C166F101C167F102C168F103C169F17B
:1049D0008EC32AF18FC32BF190C32CF191C32DF11B
:1049E00092C32EF193C32FF194C330F195C331F1EB
:1049F00096C332F197C333F10101E6EC30F05DEC80
:104A000030F000C14FF101C150F102C151F103C1B9
:104A100052F1D9EC30F099C32FF19AC330F19BC316
:104A200031F19CC332F19DC333F10101E6EC30F06A
:104A30005DEC30F000C159F101C15AF17DEC24F078
:104A400004012C0E826F94EC0EF037EF25F0118EDE
:104A50001CA002D01CAE108C1BBE02D01BA4108E5A
:104A600003018251520A02E10F8201D00F9282515A
:104A7000750A02E1108401D010948251550A02E1B6
:104A8000108601D010968351310A03E113821384FA
:104A900002D01392139403018351660A01E056D0A9
:104AA0000401660E826F94EC0EF004012C0E826FEE
:104AB00094EC0EF06CEC23F021EC30F02AC182F47F
:104AC0000401300E822794EC0EF02BC182F4040115
:104AD000300E822794EC0EF02CC182F40401300ECB
:104AE000822794EC0EF02DC182F40401300E82274F
:104AF00094EC0EF02EC182F40401300E822794EC67
:104B00000EF02FC182F40401300E822794EC0EF0D7
:104B100030C182F40401300E822794EC0EF031C1D2
:104B200082F40401300E822794EC0EF032C182F43C
:104B30000401300E822794EC0EF033C182F404019C
:104B4000300E822794EC0EF099EF29F011A003D0DB
:104B500011A401D01084078410B210EF26F010A425
:104B6000F4EF25F0BAC166F1BBC167F1BCC168F1D1
:104B7000BDC169F1BEC16AF1BFC16BF1C0C16CF1C9
:104B8000C1C16DF1C2C16EF1C3C16FF1C4C170F199
:104B9000C5C171F1C6C172F1C7C173F1C8C174F169
:104BA000C9C175F1CAC176F1CBC177F1CCC178F139
:104BB000CDC179F1CEC17AF1CFC17BF1D0C17CF109
:104BC000D1C17DF1D2C17EF1D3C17FF1D4C180F1D9
:104BD000D5C181F1D6C182F1D7C183F1D8C184F1A9
:104BE000D9C185F1FCEF25F062C166F163C167F1BF
:104BF00064C168F165C169F1BAC186F1BBC187F1D1
:104C0000BCC188F1BDC189F14BC14FF14CC150F11C
:104C10004DC151F14EC152F157C159F158C15AF12C
:104C200007940FA032EF26F0010196671FEF26F0E0
:104C300097671FEF26F098671FEF26F0996723EF1D
:104C400026F032EF26F06FEC22F096C104F197C106
:104C500005F198C106F199C107F183EC2FF003BF6C
:104C60005FEF29F06FEC22F00101000E046F000EDF
:104C7000056F010E066F000E076FB4EC2FF011A048
:104C80002AD011A228D021EC30F0296701D005D01C
:104C900004012D0E826F94EC0EF030C182F40401F9
:104CA000300E822794EC0EF031C182F40401300EF4
:104CB000822794EC0EF032C182F40401300E822778
:104CC00094EC0EF033C182F40401300E822794EC90
:104CD0000EF09EEC0EF012A8C5D012981DC01EF06A
:104CE0001E3A1E42070E1E1600011E50000AD8B4BE
:104CF000FEEF26F000011E50010AD8B48AEF26F01C
:104D000000011E50020AD8B488EF26F030EF27F0D9
:104D100030EF27F098EC30F02DC001F12EC000F1FB
:104D2000D89001330033D890013300330101630E72
:104D3000046F000E056F000E066F000E076FB4ECD7
:104D40002FF0280E046F000E056F000E066F000E88
:104D5000076F83EC2FF000C130F098EC30F02BC0DF
:104D600001F1019F019D2CC000F10101A40E046F0F
:104D7000000E056F000E066F000E076FB4EC2FF0EB
:104D800000C12FF000C104F101C105F102C106F11B
:104D900003C107F1640E006F000E016F000E026F79
:104DA000000E036F83EC2FF0050E046F000E056FED
:104DB000000E066F000E076FB4EC2FF000C104F177
:104DC00001C105F102C106F103C107F198EC30F011
:104DD00030C000F183EC2FF000C131F031C0E8FFAA
:104DE000050F305C03E78A8430EF27F031C0E8FF1D
:104DF0000A0F305C01E68A9430EF27F000C124F1FD
:104E000001C125F102C126F103C127F198EC30F070
:104E10009EEC30F01D501F0BE8CF00F10101640E35
:104E2000046F000E056F000E066F000E076F94EC06
:104E30002FF024C104F125C105F126C106F127C1D7
:104E400007F183EC2FF003BF02D08A9401D08A844B
:104E500024C100F125C101F126C102F127C103F1EE
:104E60009BEF29F000C124F101C125F102C126F117
:104E700003C127F110AE4DD0109E00C108F101C151
:104E800009F102C10AF103C10BF121EC30F030C18C
:104E9000E2F131C1E3F132C1E4F133C1E5F108C11E
:104EA00000F109C101F10AC102F10BC103F10101D5
:104EB0006C0E046F070E056F000E066F000E076F75
:104EC00083EC2FF003BF04D00101550EE66F1CD018
:104ED00008C100F109C101F10AC102F10BC103F1DE
:104EE0000101A40E046F060E056F000E066F000E82
:104EF000076F83EC2FF003BF04D001017F0EE66F34
:104F000003D00101FF0EE66F1F8E11AE5FEF29F097
:104F1000119E24C100F125C101F126C102F127C172
:104F200003F111A005D011A203D00FB05FEF29F05B
:104F300010A4A2EF27F00401750E826F94EC0EF01E
:104F4000A7EF27F00401720E826F94EC0EF00401BB
:104F50002C0E826F94EC0EF021EC30F02967B6EF46
:104F600027F00401200E826FB9EF27F004012D0E07
:104F7000826F94EC0EF030C182F40401300E82276F
:104F800094EC0EF031C182F40401300E822794ECCF
:104F90000EF004012E0E826F94EC0EF032C182F4FA
:104FA0000401300E822794EC0EF033C182F4040128
:104FB000300E822794EC0EF004016D0E826F94EC9B
:104FC0000EF004012C0E826F94EC0EF04FC100F134
:104FD00050C101F151C102F152C103F1010121ECB3
:104FE00030F0E4EC2DF00401480E826F94EC0EF0EA
:104FF00004017A0E826F94EC0EF004012C0E826F85
:1050000094EC0EF066C100F167C101F168C102F1D4
:1050100069C103F1010121EC30F0E4EC2DF0040151
:10502000630E826F94EC0EF004012C0E826F94ECF0
:105030000EF066C100F167C101F168C102F169C1FA
:1050400003F101010A0E046F000E056F000E066FDA
:10505000000E076F94EC2FF0000E046F120E056F18
:10506000000E066F000E076FB4EC2FF021EC30F04D
:105070002AC182F40401300E822794EC0EF02BC179
:1050800082F40401300E822794EC0EF02CC182F4DD
:105090000401300E822794EC0EF02DC182F404013D
:1050A000300E822794EC0EF02EC182F40401300EF3
:1050B000822794EC0EF02FC182F40401300E822777
:1050C00094EC0EF030C182F40401300E822794EC8F
:1050D0000EF004012E0E826F94EC0EF031C182F4BA
:1050E0000401300E822794EC0EF032C182F40401E8
:1050F000300E822794EC0EF033C182F40401300E9E
:10510000822794EC0EF00401730E826F94EC0EF083
:1051100004012C0E826F94EC0EF098EC30F059C123
:1051200000F15AC101F1C5EC2AF013A2E7EF28F013
:1051300004012C0E826F94EC0EF086C166F187C1DB
:1051400067F188C168F189C169F16FEC22F0010152
:10515000000E046F000E056F010E066F000E076F44
:10516000B4EC2FF021EC30F02967BCEF28F00401FB
:10517000200E826FBFEF28F004012D0E826F94EC99
:105180000EF030C182F40401300E822794EC0EF050
:1051900031C182F40401300E822794EC0EF0040138
:1051A0002E0E826F94EC0EF032C182F40401300EA8
:1051B000822794EC0EF033C182F40401300E822772
:1051C00094EC0EF004016D0E826F94EC0EF013A4BB
:1051D0000EEF29F004012C0E826F94EC0EF013AC4C
:1051E000FCEF28F00401500E826F94EC0EF0139C3B
:1051F0001398139A0EEF29F013AE09EF29F004016A
:10520000460E826F94EC0EF0139E1398139A0EEFD5
:1052100029F00401530E826F94EC0EF037B025EFA5
:1052200029F004012C0E826F94EC0EF08BB020EF6D
:1052300029F00401440E826F94EC0EF025EF29F062
:105240000401530E826F94EC0EF00FB22BEF29F095
:105250000FA05DEF29F004012C0E826F94EC0EF08C
:10526000200EF86EF76AF66A04010900F5CF82F4A1
:1052700094EC0EF00900F5CF82F494EC0EF00900E6
:10528000F5CF82F494EC0EF00900F5CF82F494ECA3
:105290000EF00900F5CF82F494EC0EF00900F5CF82
:1052A00082F494EC0EF00900F5CF82F494EC0EF049
:1052B0000900F5CF82F494EC0EF09EEC0EF00F9006
:1052C000109E12989BEF29F00401630E826F94ECFC
:1052D0000EF004012C0E826F94EC0EF0A1EC29F07C
:1052E00004012C0E826F94EC0EF014EC2AF00401F1
:1052F0002C0E826F94EC0EF090EC2AF004012C0E30
:10530000826F94EC0EF00101F80E006FCD0E016F6C
:10531000660E026F030E036FB6EC29F004012C0E2B
:10532000826F94EC0EF0A6EC2AF09EEC0EF09BEF50
:1053300029F09EEC0EF00301C26B07901092AAEFC9
:105340002CF0D8900E0E64EC0BF0E8CF00F10F0EAD
:1053500064EC0BF0E8CF01F1100E64EC0BF0E8CF39
:1053600002F1110E64EC0BF0E8CF03F10101000E25
:10537000046F000E056F010E066F000E076FB4EC90
:105380002FF021EC30F02AC182F40401300E822784
:1053900094EC0EF02BC182F40401300E822794ECC1
:1053A0000EF02CC182F40401300E822794EC0EF032
:1053B0002DC182F40401300E822794EC0EF02EC130
:1053C00082F40401300E822794EC0EF02FC182F497
:1053D0000401300E822794EC0EF030C182F40401F7
:1053E000300E822794EC0EF031C182F40401300EAD
:1053F000822794EC0EF004012E0E826F94EC0EF0D6
:1054000032C182F40401300E822794EC0EF033C1D5
:1054100082F40401300E822794EC0EF004016D0E2C
:10542000826F94EC0EF01200120E64EC0BF0E8CFD9
:1054300000F1130E64EC0BF0E8CF01F1140E64ECF4
:105440000BF0E8CF02F1150E64EC0BF0E8CF03F19E
:1054500001010A0E046F000E056F000E066F000EAC
:10546000076F94EC2FF0000E046F120E056F000E04
:10547000066F000E076FB4EC2FF021EC30F02AC15C
:1054800082F40401300E822794EC0EF02BC182F4DA
:105490000401300E822794EC0EF02CC182F404013A
:1054A000300E822794EC0EF02DC182F40401300EF0
:1054B000822794EC0EF02EC182F40401300E822774
:1054C00094EC0EF02FC182F40401300E822794EC8C
:1054D0000EF030C182F40401300E822794EC0EF0FD
:1054E00004012E0E826F94EC0EF031C182F404019F
:1054F000300E822794EC0EF032C182F40401300E9B
:10550000822794EC0EF033C182F40401300E82271E
:1055100094EC0EF00401730E826F94EC0EF0120006
:105520000A0E64EC0BF0E8CF00F10B0E64EC0BF00C
:10553000E8CF01F10C0E64EC0BF0E8CF02F10D0E98
:1055400064EC0BF0E8CF03F1C5EF2AF0060E64EC33
:105550000BF0E8CF00F1070E64EC0BF0E8CF01F19F
:10556000080E64EC0BF0E8CF02F1090E64EC0BF0CE
:10557000E8CF03F1C5EF2AF0010198EC30F0078481
:1055800057C100F158C101F107940101E80E046F01
:10559000800E056F000E066F000E076F94EC2FF063
:1055A000000E046F040E056F000E066F000E076FED
:1055B000B4EC2FF0880E046F130E056F000E066F0B
:1055C000000E076F83EC2FF00A0E046F000E056FBC
:1055D000000E066F000E076FB4EC2FF021EC30F0D8
:1055E00001012967F9EF2AF00401200E826FFCEF18
:1055F0002AF004012D0E826F94EC0EF030C182F47B
:105600000401300E822794EC0EF031C182F40401C3
:10561000300E822794EC0EF032C182F40401300E79
:10562000822794EC0EF004012E0E826F94EC0EF0A3
:1056300033C182F40401300E822794EC0EF0040191
:10564000430E826F94EC0EF0120087C32AF188C3D8
:105650002BF189C32CF18AC32DF18BC32EF18CC39E
:105660002FF18DC330F18EC331F190C332F191C36C
:1056700033F10101296BE6EC30F05DEC30F0010113
:10568000000E046F000E056F010E066F000E076F0F
:1056900094EC2FF00E0E0C6E00C10BF04DEC0BF0E5
:1056A0000F0E0C6E01C10BF04DEC0BF0100E0C6EDA
:1056B00002C10BF04DEC0BF0110E0C6E03C10BF0A0
:1056C0004DEC0BF004017A0E826F94EC0EF00401A5
:1056D0002C0E826F94EC0EF00401350E826F94EC68
:1056E0000EF004012C0E826F94EC0EF0A1EC29F068
:1056F00045EF22F087C32AF188C32BF189C32CF12F
:105700008AC32DF18BC32EF18CC32FF18DC330F1E1
:105710008EC331F190C332F191C333F10101296B92
:10572000E6EC30F05DEC30F0880E046F130E056F80
:10573000000E066F000E076F88EC2FF0000E046F4E
:10574000040E056F000E066F000E076F94EC2FF02D
:105750000101E80E046F800E056F000E066F000E4B
:10576000076FB4EC2FF00A0E0C6E00C10BF04DEC7D
:105770000BF00B0E0C6E01C10BF04DEC0BF00C0E90
:105780000C6E02C10BF04DEC0BF00D0E0C6E03C154
:105790000BF04DEC0BF004017A0E826F94EC0EF0DE
:1057A00004012C0E826F94EC0EF00401360E826F11
:1057B00094EC0EF004012C0E826F94EC0EF090EC41
:1057C0002AF045EF22F087C32AF188C32BF189C361
:1057D0002CF18AC32DF18BC32EF18CC32FF18DC315
:1057E00030F18FC331F190C332F191C333F1010134
:1057F000E6EC30F05DEC30F0000E046F120E056F39
:10580000000E066F000E076F94EC2FF001010A0ED8
:10581000046F000E056F000E066F000E076FB4ECEC
:105820002FF0120E0C6E00C10BF04DEC0BF0130EAE
:105830000C6E01C10BF04DEC0BF0140E0C6E02C19E
:105840000BF04DEC0BF0150E0C6E03C10BF04DEC94
:105850000BF004017A0E826F94EC0EF004012C0E12
:10586000826F94EC0EF00401370E826F94EC0EF010
:1058700004012C0E826F94EC0EF014EC2AF045EF2C
:1058800022F087C32AF188C32BF189C32CF18AC384
:105890002DF18BC32EF18CC32FF18DC330F18EC34C
:1058A00031F190C332F191C333F10101296BE6EC80
:1058B00030F05DEC30F0880E046F130E056F000EB3
:1058C000066F000E076F88EC2FF0000E046F040EB9
:1058D000056F000E066F000E076F94EC2FF00101AC
:1058E000E80E046F800E056F000E066F000E076F46
:1058F000B4EC2FF0060E0C6E00C10BF04DEC0BF06B
:10590000070E0C6E01C10BF04DEC0BF0080E0C6E87
:1059100002C10BF04DEC0BF0090E0C6E03C10BF045
:105920004DEC0BF004017A0E826F94EC0EF0040142
:105930002C0E826F94EC0EF00401380E826F94EC02
:105940000EF004012C0E826F94EC0EF0A6EC2AF0FF
:1059500045EF22F007A81DEF2DF00101800E006F2A
:105960001A0E016F060E026F000E036F4BC104F199
:105970004CC105F14DC106F14EC107F183EC2FF08A
:1059800003BF63EF2DF0DEEC2DF04BC100F14CC1F5
:1059900001F14DC102F14EC103F1078290EC2EF0EE
:1059A00018C104F119C105F11AC106F11BC107F1B3
:1059B000F80E006FCD0E016F660E026F030E036FBF
:1059C00083EC2FF00E0E0C6E00C10BF04DEC0BF0C3
:1059D0000F0E0C6E01C10BF04DEC0BF0100E0C6EA7
:1059E00002C10BF04DEC0BF0110E0C6E03C10BF06D
:1059F0004DEC0BF00784010198EC30F057C100F139
:105A000058C101F107940A0E0C6E00C10BF04DEC69
:105A10000BF00B0E0C6E01C10BF04DEC0BF00C0EED
:105A20000C6E02C10BF04DEC0BF00D0E0C6E03C1B1
:105A30000BF04DEC0BF063EF2DF007AA63EF2DF0A8
:105A40000784010198EC30F057C100F158C101F111
:105A50000794060E0C6E00C10BF04DEC0BF0070E18
:105A60000C6E01C10BF04DEC0BF0080E0C6E02C178
:105A70000BF04DEC0BF0090E0C6E03C10BF04DEC6E
:105A80000BF0078462C100F163C101F164C102F14E
:105A900065C103F10794120E0C6E00C10BF04DECC2
:105AA0000BF0130E0C6E01C10BF04DEC0BF0140E4D
:105AB0000C6E02C10BF04DEC0BF0150E0C6E03C119
:105AC0000BF04DEC0BF00798079A040180518119F7
:105AD0007F0B0DE09EA8FED714EE00F081517F0BE6
:105AE000E126E750812B0F01AD6E65EF2DF005012A
:105AF0002F51000AD8B4A6EF2DF081BA8BEF2DF00C
:105B000015B2A6EF2DF005012F51010AD8B4A4EF6C
:105B10002DF09DEF2DF005012F51000AD8B45DEF57
:105B200038F005012F51010AD8B4A4EF2DF000017F
:105B30001650050AD8B45DEF38F081B8A6EF2DF005
:105B4000E1EC31F0DFEC32F0F6EC37F0C2EF0DF0C3
:105B500018C100F119C101F11AC102F11BC103F111
:105B6000000E046F000E056F010E066F000E076F2A
:105B7000B4EC2FF029A1D3EF2DF02051D8B4D3EFFE
:105B80002DF018C100F119C101F11AC102F11BC1B8
:105B900003F1000E046F000E056F0A0E066F000E73
:105BA000076FB4EC2FF012000101045100130551EE
:105BB0000113065102130751031312000101186B60
:105BC000196B1A6B1B6B12002AC182F40401300E90
:105BD000822794EC0EF02BC182F40401300E822750
:105BE00094EC0EF02CC182F40401300E822794EC68
:105BF0000EF02DC182F40401300E822794EC0EF0D9
:105C00002EC182F40401300E822794EC0EF02FC1D5
:105C100082F40401300E822794EC0EF030C182F43D
:105C20000401300E822794EC0EF031C182F404019D
:105C3000300E822794EC0EF032C182F40401300E53
:105C4000822794EC0EF033C182F40401300E8227D7
:105C500094EC0EF012002FC182F40401300E822762
:105C600094EC0EF030C182F40401300E822794ECE3
:105C70000EF031C182F40401300E822794EC0EF054
:105C800032C182F40401300E822794EC0EF033C14D
:105C900082F40401300E822794EC0EF01200060EFE
:105CA000216E060E226E060E236E212E55EF2EF06B
:105CB000222E55EF2EF0232E55EF2EF08B84020E60
:105CC000216E020E226E020E236E212E65EF2EF043
:105CD000222E65EF2EF0232E65EF2EF08B9412000E
:105CE000FF0E226E22C023F0030E216E8B84212E24
:105CF00076EF2EF0030E216E232E76EF2EF08B948E
:105D000022C023F0030E216E212E84EF2EF0030E0D
:105D1000216E233E84EF2EF0222E72EF2EF0120021
:105D20000101005305E1015303E1025301E1002B9E
:105D300053EC2FF098EC30F03951006F3A51016F6D
:105D4000420E046F4B0E056F000E066F000E076FBC
:105D500094EC2FF000C104F101C105F102C106F17C
:105D600003C107F118C100F119C101F11AC102F113
:105D70001BC103F107B2C1EF2EF088EC2FF0C3EF87
:105D80002EF083EC2FF000C118F101C119F102C10E
:105D90001AF103C11BF1120098EC30F059C100F167
:105DA0005AC101F1060E64EC0BF0E8CF04F1070EC6
:105DB00064EC0BF0E8CF05F1080E64EC0BF0E8CFD3
:105DC00006F1090E64EC0BF0E8CF07F183EC2FF03D
:105DD00000C124F101C125F102C126F103C127F15F
:105DE000290E046F000E056F000E066F000E076F80
:105DF00094EC2FF0EE0E046F430E056F000E066F4D
:105E0000000E076F88EC2FF024C104F125C105F1C5
:105E100026C106F127C107F194EC2FF000C11CF157
:105E200001C11DF102C11EF103C11FF1120E64EC8C
:105E30000BF0E8CF04F1130E64EC0BF0E8CF05F1A2
:105E4000140E64EC0BF0E8CF06F1150E64EC0BF0C9
:105E5000E8CF07F10D0E006F000E016F000E026F0C
:105E6000000E036F94EC2FF0180E046F000E056FF8
:105E7000000E066F000E076FB4EC2FF01CC104F18A
:105E80001DC105F11EC106F11FC107F188EC2FF0FD
:105E90006A0E046F2A0E056F000E066F000E076F64
:105EA00083EC2FF01200BF0EFA6E200E3A6F396BA2
:105EB000D8900037013702370337D8B064EF2FF09E
:105EC0003A2F59EF2FF039073A070353D8B412008D
:105ED0000331070B80093F6F03390F0B010F396F37
:105EE00080EC5FF0406F390580EC5FF0405D405F13
:105EF000396B3F33D8B0392739333FA979EF2FF0C9
:105F00004051392712000101BDEC30F0D8B0120029
:105F1000010103510719346F80EC30F0D89007511C
:105F2000031934AF800F12000101346BA4EC30F080
:105F3000D8A0BAEC30F0D8B012008FEC30F098EC6A
:105F400030F01F0E366FD0EC30F00B35D8B080EC4F
:105F500030F0D8A00335D8B01200362FA3EF2FF0C1
:105F600034B1A7EC30F012000101346B045105117B
:105F7000061107110008D8A0A4EC30F0D8A0BAECA4
:105F800030F0D8B01200086B096B0A6B0B6BD0ECC9
:105F900030F01F0E366FD0EC30F007510B5DD8A4F7
:105FA000DEEF2FF006510A5DD8A4DEEF2FF0055189
:105FB000095DD8A4DEEF2FF00451085DD8A0F1EF01
:105FC0002FF00451085F0551D8A0053D095F065127
:105FD000D8A0063D0A5F0751D8A0073D0B5FD890B7
:105FE0000081362FCBEF2FF034B1A7EC30F0346BBB
:105FF000A4EC30F0D890D4EC30F007510B5DD8A46D
:106000000EEF30F006510A5DD8A40EEF30F00551C6
:10601000095DD8A40EEF30F00451085DD8A01DEF43
:1060200030F0003F1DEF30F0013F1DEF30F0023F38
:106030001DEF30F0032BD8B4120034B1A7EC30F0D0
:1060400012000101346BA4EC30F0D8B01200D9EC8E
:1060500030F0200E366F003701370237033711EE6C
:1060600033F00A0E376FE7360A0EE75CD8B0E76EFA
:10607000E552372F33EF30F0362F2BEF30F034B1BD
:106080002981D8901200D9EC30F0200E366F0037FD
:1060900001370237033711EE33F00A0E376FE73658
:1060A0000A0EE75CD8B0E76EE552372F4FEF30F0BD
:1060B000362F47EF30F0D890120001010A0E346FEE
:1060C000200E366F11EE29F03451376F0A0ED8903A
:1060D000E652D8B0E726E732372F68EF30F00333C7
:1060E000023301330033362F62EF30F0E750FF0FF9
:1060F000D8A00335D8B0120029B1A7EC30F01200B7
:10610000045100270551D8B0053D01270651D8B0EC
:10611000063D02270751D8B0073D03271200005162
:10612000086F0151096F02510A6F03510B6F120082
:106130000101006B016B026B036B12000101046B28
:10614000056B066B076B12000335D8A012000351D4
:10615000800B001F011F021F031F003FB7EF30F02D
:10616000013FB7EF30F0023FB7EF30F0032B342B95
:10617000032512000735D8A012000751800B041F19
:10618000051F061F071F043FCDEF30F0053FCDEF81
:1061900030F0063FCDEF30F0072B342B07251200EF
:1061A0000037013702370337083709370A370B370B
:1061B00012000101296B2A6B2B6B2C6B2D6B2E6B44
:1061C0002F6B306B316B326B336B120001012A5134
:1061D0000F0B2A6F2B510F0B2B6F2C510F0B2C6FAA
:1061E0002D510F0B2D6F2E510F0B2E6F2F510F0BAB
:1061F0002F6F30510F0B306F31510F0B316F325108
:106200000F0B326F33510F0B336F120000C124F1AB
:1062100001C125F102C126F103C127F104C100F13A
:1062200005C101F106C102F107C103F124C104F166
:1062300025C105F126C106F127C107F1120010A8FA
:1062400006D08994000EC76E220EC66E05D08984D2
:10625000000EC76E220EC66E050EE82EFED7120087
:1062600010A802D0898401D08994050EE82EFED7AB
:1062700012001FEC31F09E96C69E000EC96EFF0EF6
:106280009EB602D0E82EFCD79E96C69E000EC96E22
:10629000FF0E9EB602D0E82EFCD7C9CFAFF59E9672
:1062A000C69E000EC96EFF0E9EB602D0E82EFCD729
:1062B000C9CFB0F59E96C69E000EC96EFF0E9EB663
:1062C00002D0E82EFCD7C9CFB1F59E96C69E000E2F
:1062D000C96EFF0E9EB602D0E82EFCD7C9CFB2F52C
:1062E0009E96C69E000EC96EFF0E9EB602D0E82E88
:1062F000FCD7C9CFB3F59E96C69E000EC96EFF0EA1
:106300009EB602D0E82EFCD7C9CFB4F59E96C69EA5
:10631000000EC96EFF0E9EB602D0E82EFCD7C9CF84
:10632000B5F530EC31F012001FEC31F09E96C69EB0
:10633000800EC96EFF0E9EB602D0E82EFCD79E9648
:10634000C69EAFC5C9FFFF0E9EB602D0E82EFCD791
:106350009E96C69EB0C5C9FFFF0E9EB602D0E82E1F
:10636000FCD79E96C69EB1C5C9FFFF0E9EB602D051
:10637000E82EFCD79E96C69EB2C5C9FFFF0E9EB6FC
:1063800002D0E82EFCD79E96C69EB3C5C9FFFF0E6D
:106390009EB602D0E82EFCD79E96C69EB4C5C9FF15
:1063A000FF0E9EB602D0E82EFCD79E96C69EB5C5BF
:1063B000C9FFFF0E9EB602D0E82EFCD730EC31F0BC
:1063C00012001FEC31F09E96C69E070EC96EFF0E9E
:1063D0009EB602D0E82EFCD79E96C69E000EC96ED1
:1063E000FF0E9EB602D0E82EFCD7C9CFAFF59E9621
:1063F000C69E000EC96EFF0E9EB602D0E82EFCD7D8
:10640000C9CFB0F59E96C69E000EC96EFF0E9EB611
:1064100002D0E82EFCD7C9CFB1F59E96C69E000EDD
:10642000C96EFF0E9EB602D0E82EFCD7C9CFB2F5DA
:1064300030EC31F01FEC31F09E96C69E25C0C9FFAE
:10644000FF0E9EB602D0E82EFCD79E96C69E000E8A
:10645000C96EFF0E9EB602D0E82EFCD7C9CFB6F5A6
:1064600030EC31F012001FEC31F09E96C69E870E84
:10647000C96EFF0E9EB602D0E82EFCD79E96C69E31
:10648000AFC5C9FFFF0E9EB602D0E82EFCD79E9680
:10649000C69EB0C5C9FFFF0E9EB602D0E82EFCD73F
:1064A0009E96C69EB1C5C9FFFF0E9EB602D0E82ECD
:1064B000FCD79E96C69EB2C5C9FFFF0E9EB602D0FF
:1064C000E82EFCD730EC31F01FEC31F09E96C69EE2
:1064D00026C0C9FFFF0E9EB602D0E82EFCD79E96BE
:1064E000C69EB6C5C9FFFF0E9EB602D0E82EFCD7E9
:1064F00030EC31F012001FEC31F09E96C69E870EF4
:10650000C96EFF0E9EB602D0E82EFCD79E96C69EA0
:10651000000EC96EFF0E9EB602D0E82EFCD79E96E6
:10652000C69E800EC96EFF0E9EB602D0E82EFCD726
:106530009E96C69E800EC96EFF0E9EB602D0E82EB5
:10654000FCD79E96C69E800EC96EFF0E9EB602D0E8
:10655000E82EFCD730EC31F012001FEC31F09E96A3
:10656000C69E870EC96EFF0E9EB602D0E82EFCD7DF
:106570009E96C69E000EC96EFF0E9EB602D0E82EF5
:10658000FCD79E96C69E000EC96EFF0E9EB602D028
:10659000E82EFCD79E96C69E800EC96EFF0E9EB654
:1065A00002D0E82EFCD79E96C69E800EC96EFF0EC6
:1065B0009EB602D0E82EFCD730EC31F0120010A8C5
:1065C00017D01FEC31F09E96C69E8F0EC96EFF0E3F
:1065D0009EB602D0E82EFCD79E96C69E000EC96ECF
:1065E000FF0E9EB602D0E82EFCD730EC31F0120040
:1065F000E1EC31F0120010A82DD01FEC31F09E9686
:10660000C69E26C0C9FFFF0E9EB602D0E82EFCD75C
:106610009E96C69E450EC96EFF0E9EB602D0E82E0F
:10662000FCD730EC31F01FEC31F09E96C69E8F0EF9
:10663000C96EFF0E9EB602D0E82EFCD79E96C69E6F
:10664000000EC96EFF0E9EB602D0E82EFCD730ECCD
:1066500031F012001FEC31F09E96C69E26C0C9FF95
:10666000FF0E9EB602D0E82EFCD79E96C69E010E67
:10667000C96EFF0E9EB602D0E82EFCD730EC31F08A
:106680001FEC31F09E96C69E910EC96EFF0E9EB60F
:1066900002D0E82EFCD79E96C69EA50EC96EFF0EB0
:1066A0009EB602D0E82EFCD730EC31F012001FEC81
:1066B00031F09E96C69E26C0C9FFFF0E9EB602D040
:1066C000E82EFCD79E96C69E810EC96EFF0E9EB622
:1066D00002D0E82EFCD730EC31F012001FEC31F084
:1066E0009E96C69E26C0C9FFFF0E9EB602D0E82E1B
:1066F000FCD79E96C69E010EC96EFF0E9EB602D0B6
:10670000E82EFCD730EC31F012001FEC31F09E96F1
:10671000C69E910EC96EFF0E9EB602D0E82EFCD723
:106720009E96C69EA50EC96EFF0E9EB602D0E82E9E
:10673000FCD730EC31F012001FEC31F09E96C69E73
:10674000910EC96EFF0E9EB602D0E82EFCD79E9623
:10675000C69E000EC96EFF0E9EB602D0E82EFCD774
:1067600030EC31F012000501256B266B276B286B8E
:10677000899A400EC76E200EC66E9E96C69E030E68
:10678000C96EFF0E9EB602D0E82EFCD79E96C69E1E
:1067900027C5C9FFFF0E9EB602D0E82EFCD79E96F5
:1067A000C69E26C5C9FFFF0E9EB602D0E82EFCD7B6
:1067B0009E96C69E25C5C9FFFF0E9EB602D0E82E46
:1067C000FCD79E96C69EC952FF0E9EB602D0E82EFA
:1067D000FCD7898A0F01C950FF0A01E112000501A7
:1067E0002E51130A05E005012E51170A0CE0120084
:1067F0000501F00E256FFF0E266F0F0E276F000E9E
:10680000286F0CEF34F00501F00E256FFF0E266F98
:10681000FF0E276F000E286F899A400EC76E200E5C
:10682000C66E9E96C69E030EC96EFF0E9EB602D021
:10683000E82EFCD79E96C69E27C5C9FFFF0E9EB6C2
:1068400002D0E82EFCD79E96C69E26C5C9FFFF0E35
:106850009EB602D0E82EFCD79E96C69E25C5C9FFDF
:10686000FF0E9EB602D0E82EFCD79E96C69EC95259
:10687000FF0E9EB602D0E82EFCD7898A0F01C950C0
:10688000FF0A1DE005012E51130A05E005012E51F6
:10689000170A0BE012000501000E256F000E266F8F
:1068A000100E276F000E286F12000501000E256FD5
:1068B000000E266F000E276F010E286F12000501D3
:1068C000256B266B276B286B05012E51130A05E0FB
:1068D00005012E51170A0CE012000501000E216F70
:1068E000000E226F080E236F000E246F81EF34F02C
:1068F0000501000E216F000E226F800E236F000E27
:10690000246F21C500F122C501F123C502F124C580
:1069100003F125C504F126C505F127C506F128C5F3
:1069200007F1D4EC2DF000C125F501C126F502C117
:1069300027F503C128F5899A400EC76E200EC66E52
:106940009E96C69E030EC96EFF0E9EB602D0E82E1E
:10695000FCD79E96C69E27C5C9FFFF0E9EB602D0E5
:10696000E82EFCD79E96C69E26C5C9FFFF0E9EB692
:1069700002D0E82EFCD79E96C69E25C5C9FFFF0E05
:106980009EB602D0E82EFCD79E96C69EC952FF0E38
:106990009EB602D0E82EFCD7898AC950FF0A08E1CA
:1069A00004C125F505C126F506C127F507C128F55F
:1069B000D890050124332333223321332151F00BA6
:1069C000216F05012167ECEF34F02267ECEF34F022
:1069D0002367ECEF34F0246781EF34F00501100EEB
:1069E0002527E86A2623E86A2723E86A2823120075
:1069F000E86A05012E51130A06E005012E51170A17
:106A00000BE0020E120005012851000A03E1275194
:106A1000F00B07E0010E120005012851000A01E009
:106A2000010E120029C500F12AC501F12BC502F1A2
:106A30002CC503F125C504F126C505F127C506F1CE
:106A400028C507F183EC2FF003BF1200F8EC34F0F7
:106A5000D8A48AEF35F0899A400EC76E200EC66E14
:106A60009E96C69E060EC96EFF0E9EB602D0E82EFA
:106A7000FCD7898A899A9E96C69E020EC96EFF0E21
:106A80009EB602D0E82EFCD79E96C69E27C5C9FFAB
:106A9000FF0E9EB602D0E82EFCD79E96C69E26C557
:106AA000C9FFFF0E9EB602D0E82EFCD79E96C69E6A
:106AB00025C5C9FFFF0E9EB602D0E82EFCD79E96D4
:106AC000C69E000EC96EFF0E9EB602D0E82EFCD701
:106AD000898A899A9E96C69E050EC96EFF0E9EB63D
:106AE00002D0E82EFCD79E96C69EC952FF0E9EB6D7
:106AF00002D0E82EFCD7C9B073EF35F0898A0501C2
:106B0000100E2527E86A2623E86A2723E86A282347
:106B100012EF35F01200899A400EC76E200EC66E35
:106B20009E96C69E060EC96EFF0E9EB602D0E82E39
:106B3000FCD7898A899A9E96C69EC70EC96EFF0E9B
:106B40009EB602D0E82EFCD7898A0501256B266BFC
:106B5000276B286B1200899A400EC76E200EC66EF6
:106B60009E96C69E050EC96EFF0E9EB602D0E82EFA
:106B7000FCD79E96C69EC952FF0E9EB602D0E82E46
:106B8000FCD7C9CF37F5898A1200899A400EC76EA3
:106B9000200EC66E9E96C69EB90EC96EFF0E9EB69C
:106BA00002D0E82EFCD7898A1200899A400EC76E5F
:106BB000200EC66E9E96C69EAB0EC96EFF0E9EB68A
:106BC00002D0E82EFCD7898AFF0EE82EFED71200ED
:106BD000F8EC34F0D8A41200899A400EC76E200E4B
:106BE000C66E9E96C69E030EC96EFF0E9EB602D05E
:106BF000E82EFCD79E96C69E27C5C9FFFF0E9EB6FF
:106C000002D0E82EFCD79E96C69E26C5C9FFFF0E71
:106C10009EB602D0E82EFCD79E96C69E25C5C9FF1B
:106C2000FF0E9EB602D0E82EFCD79E96C69EC95295
:106C3000FF0E9EB602D0E82EFCD7898A0F01C950FC
:106C4000FF0AD8A467EF37F00501FE0E376F050184
:106C5000FF0E536FFF0E546FFF0E556FFF0E566FF2
:106C600015A63799158639EC31F0AFC538F5B0C5A2
:106C700039F5B1C53AF5B2C53BF5B3C53CF5B4C578
:106C80003DF5B5C53EF50784BAC166F1BBC167F1F4
:106C9000BCC168F1BDC169F14BC14FF14CC150F1AC
:106CA0004DC151F14EC152F157C159F158C15AF17C
:106CB00000011650010AD8B46CEF36F000011650EE
:106CC000020AD8B491EF36F000011650040AD8B485
:106CD000B6EF36F067EF37F00501476B486B496B4D
:106CE0004A6B05014B6B4C6B4D6B4E6B05014F6B4B
:106CF000506B516B526B8BA0379B6FEC22F000C135
:106D0000DAF101C1DBF102C1DCF103C1DDF100C147
:106D10003FF501C140F502C141F503C142F5D5EF90
:106D200036F00501476B486B496B4A6B05014B6BAD
:106D30004C6B4D6B4E6B05014F6B506B516B526B37
:106D40006FEC22F000C1DAF101C1DBF102C1DCF12C
:106D500003C1DDF16CEC23F000C147F501C148F53A
:106D600002C149F503C14AF567EF37F0379BDAC135
:106D70003FF5DBC140F5DCC141F5DDC142F56FEC0B
:106D800022F000C14BF501C14CF502C14DF503C124
:106D90004EF56CEC23F000C14FF501C150F502C176
:106DA00051F503C152F5D5EF36F005016167E0EF0B
:106DB00036F06267E0EF36F06367E0EF36F0646765
:106DC000E4EF36F0F9EF36F0DAC100F1DBC101F1A2
:106DD000DCC102F1DDC103F161C504F162C505F159
:106DE00063C506F164C507F183EC2FF003BF67EFBD
:106DF00037F059C143F55AC144F5B9C545F5050108
:106E0000110E326F899A400EC76E200EC66E9E9686
:106E1000C69E060EC96EFF0E9EB602D0E82EFCD7A7
:106E2000898A899A9E96C69E020EC96EFF0E9EB6EC
:106E300002D0E82EFCD79E96C69E27C5C9FFFF0E3E
:106E40009EB602D0E82EFCD79E96C69E26C5C9FFE8
:106E5000FF0E9EB602D0E82EFCD79E96C69E25C594
:106E6000C9FFFF0E9EB602D0E82EFCD725EE37F004
:106E7000322F02D047EF37F09E96C69EDECFC9FF75
:106E8000FF0E9EB602D0E82EFCD738EF37F0898A85
:106E9000899A9E96C69E050EC96EFF0E9EB602D0BA
:106EA000E82EFCD79E96C69EC952FF0E9EB602D013
:106EB000E82EFCD7C9B052EF37F0898A0501100ED1
:106EC0002527E86A2623E86A2723E86A28231590FD
:106ED0000794120021C500F122C501F123C502F17A
:106EE00024C503F1899A400EC76E200EC66E9E9689
:106EF000C69E0B0EC96EFF0E9EB602D0E82EFCD7C2
:106F00009E96C69E02C1C9FFFF0E9EB602D0E82E15
:106F1000FCD79E96C69E01C1C9FFFF0E9EB602D049
:106F2000E82EFCD79E96C69E00C1C9FFFF0E9EB6F6
:106F300002D0E82EFCD79E96C69EC952FF0E9EB682
:106F400002D0E82EFCD725EE37F00501100E326F87
:106F50009E96C69EC952FF0E9EB602D0E82EFCD762
:106F6000C9CFDEFF322FA8EF37F0898A1200899A45
:106F7000400EC76E200EC66E9E96C69E900EC96EBF
:106F8000FF0E9EB602D0E82EFCD79E96C69E000E3F
:106F9000C96EFF0E9EB602D0E82EFCD79E96C69E06
:106FA000000EC96EFF0E9EB602D0E82EFCD79E964C
:106FB000C69E000EC96EFF0E9EB602D0E82EFCD70C
:106FC0009E96C69EC952FF0E9EB602D0E82EFCD7F2
:106FD000C9CF2DF59E96C69EC952FF0E9EB602D011
:106FE000E82EFCD7C9CF2EF5898A120039EC31F092
:106FF00005012F51010A5FE005012F51020A16E039
:1070000005012F51030A19E005012F51040A24E05C
:1070100005012F51050A2BE005012F51060A39E021
:1070200005012F51070A3FE05BEF38F0602F59EF61
:1070300038F05FC560F55BEF38F0B0C500F10101D5
:107040000F0E001701010051000A35E00101005147
:10705000050A31E059EF38F0B0C500F101010F0E1B
:10706000001701010051000A26E059EF38F0050130
:10707000B051000A20E00501B051150A1CE00501DD
:10708000B051300A18E00501B051450A14E059EF3B
:1070900038F00501B051000A0EE00501B051300A88
:1070A0000AE059EF38F00501B051000A04E059EF49
:1070B00038F015901200158012008B904FEC2EF0D6
:1070C000B9C5E8FFD70802E34FEC2EF0B9C5E8FFD9
:1070D000C80802E34FEC2EF0B9C5E8FFB90802E397
:1070E0004FEC2EF0B9C5E8FFAA0802E34FEC2EF0F2
:1070F000B9C5E8FF9B0802E34FEC2EF0C5EC35F074
:10710000F29CF29E8B94C69AC2909482948C720EDA
:10711000D36ED3A4FED789968A909390F29AF29474
:107120009D909E909D929E92F298F292DFEC32F0AA
:10713000FF0EE8CF00F0E82EFED7002EFCD7F2902D
:10714000F286815081A8A7EF38F0F29E0300700EFE
:10715000D36EF296F2901584038070EC2EF09AEFC5
:027160000BF032
:10BF0000E844F926000C160C2B0C3F0C520C640C68
:10BF1000760C860C960CA50CB30CC10CCF0CDC0C6B
:06BF2000E80CF40C000C1B
:0200000400F00A
:0100C800FE39
:00000001FF
